Archive member included because of file (symbol)

C:/Program Files/Microchip/MPLAB C32 Suite/bin/../lib/gcc/pic32mx/3.4.4/size\libgcc.a(_udivdi3.o)
                              ..\Microchip\TCPIP Stack\Objects - TCPIP Demo App-C32\TCPPerformanceTest.o (__udivdi3)
C:/Program Files/Microchip/MPLAB C32 Suite/bin/../lib/gcc/pic32mx/3.4.4/../../../../pic32mx/lib/size\libc.a(memcmp.o)
                              Objects - TCPIP Demo App-C32\CustomHTTPApp.o (memcmp)
C:/Program Files/Microchip/MPLAB C32 Suite/bin/../lib/gcc/pic32mx/3.4.4/../../../../pic32mx/lib/size\libc.a(memcpy.o)
                              Objects - TCPIP Demo App-C32\MainDemo.o (memcpy)
C:/Program Files/Microchip/MPLAB C32 Suite/bin/../lib/gcc/pic32mx/3.4.4/../../../../pic32mx/lib/size\libc.a(memset.o)
                              Objects - TCPIP Demo App-C32\CustomHTTPApp.o (memset)
C:/Program Files/Microchip/MPLAB C32 Suite/bin/../lib/gcc/pic32mx/3.4.4/../../../../pic32mx/lib/size\libc.a(strcmp.o)
                              Objects - TCPIP Demo App-C32\CustomHTTPApp.o (strcmp)
C:/Program Files/Microchip/MPLAB C32 Suite/bin/../lib/gcc/pic32mx/3.4.4/../../../../pic32mx/lib/size\libc.a(strcpy.o)
                              Objects - TCPIP Demo App-C32\MainDemo.o (strcpy)
C:/Program Files/Microchip/MPLAB C32 Suite/bin/../lib/gcc/pic32mx/3.4.4/../../../../pic32mx/lib/size\libc.a(strlen.o)
                              Objects - TCPIP Demo App-C32\MainDemo.o (strlen)
C:/Program Files/Microchip/MPLAB C32 Suite/bin/../lib/gcc/pic32mx/3.4.4/../../../../pic32mx/lib/size\libc.a(general-exception.o)
                              C:/Program Files/Microchip/MPLAB C32 Suite/bin/../lib/gcc/pic32mx/3.4.4/../../../../pic32mx/lib/size/crt0.o (_general_exception_context)
C:/Program Files/Microchip/MPLAB C32 Suite/bin/../lib/gcc/pic32mx/3.4.4/../../../../pic32mx/lib/size\libc.a(strcat.o)
                              Objects - TCPIP Demo App-C32\PingDemo.o (strcat)
C:/Program Files/Microchip/MPLAB C32 Suite/bin/../lib/gcc/pic32mx/3.4.4/../../../../pic32mx/lib/size\libc.a(strncmp.o)
                              Objects - TCPIP Demo App-C32\CustomSNMPApp.o (strncmp)
C:/Program Files/Microchip/MPLAB C32 Suite/bin/../lib/gcc/pic32mx/3.4.4/../../../../pic32mx/lib/size\libc.a(strchr.o)
                              ..\Microchip\TCPIP Stack\Objects - TCPIP Demo App-C32\SMTP.o (strchr)
C:/Program Files/Microchip/MPLAB C32 Suite/bin/../lib/gcc/pic32mx/3.4.4/../../../../pic32mx/lib/size\libc.a(strstr.o)
                              ..\Microchip\TCPIP Stack\Objects - TCPIP Demo App-C32\SMTP.o (strstr)
C:/Program Files/Microchip/MPLAB C32 Suite/bin/../lib/gcc/pic32mx/3.4.4/../../../../pic32mx/lib/size\libc.a(exit.o)
                              C:/Program Files/Microchip/MPLAB C32 Suite/bin/../lib/gcc/pic32mx/3.4.4/../../../../pic32mx/lib/size/crt0.o (exit)
C:/Program Files/Microchip/MPLAB C32 Suite/bin/../lib/gcc/pic32mx/3.4.4/../../../../pic32mx/lib/size\libc.a(rand.o)
                              ..\Microchip\TCPIP Stack\Objects - TCPIP Demo App-C32\Helpers.o (rand)
C:/Program Files/Microchip/MPLAB C32 Suite/bin/../lib/gcc/pic32mx/3.4.4/../../../../pic32mx/lib/size\libc.a(atol.o)
                              Objects - TCPIP Demo App-C32\CustomHTTPApp.o (atol)
C:/Program Files/Microchip/MPLAB C32 Suite/bin/../lib/gcc/pic32mx/3.4.4/../../../../pic32mx/lib/size\libc.a(atoi.o)
                              ..\Microchip\TCPIP Stack\Objects - TCPIP Demo App-C32\SMTP.o (atoi)
C:/Program Files/Microchip/MPLAB C32 Suite/bin/../lib/gcc/pic32mx/3.4.4/../../../../pic32mx/lib/size\libc.a(strtol.o)
                              C:/Program Files/Microchip/MPLAB C32 Suite/bin/../lib/gcc/pic32mx/3.4.4/../../../../pic32mx/lib/size\libc.a(atol.o) (strtol)
C:/Program Files/Microchip/MPLAB C32 Suite/bin/../lib/gcc/pic32mx/3.4.4/../../../../pic32mx/lib/size\libc.a(_iobdata.o)
                              C:/Program Files/Microchip/MPLAB C32 Suite/bin/../lib/gcc/pic32mx/3.4.4/../../../../pic32mx/lib/size\libc.a(exit.o) (_libc_data)
C:/Program Files/Microchip/MPLAB C32 Suite/bin/../lib/gcc/pic32mx/3.4.4/../../../../pic32mx/lib/size\libc.a(_iobfuncs.o)
                              C:/Program Files/Microchip/MPLAB C32 Suite/bin/../lib/gcc/pic32mx/3.4.4/../../../../pic32mx/lib/size\libc.a(_iobdata.o) (_filbuf_simple)
C:/Program Files/Microchip/MPLAB C32 Suite/bin/../lib/gcc/pic32mx/3.4.4/../../../../pic32mx/lib/size\libc.a(stubs.o)
                              C:/Program Files/Microchip/MPLAB C32 Suite/bin/../lib/gcc/pic32mx/3.4.4/../../../../pic32mx/lib/size\libc.a(exit.o) (pthread_mutex_lock)
C:/Program Files/Microchip/MPLAB C32 Suite/bin/../lib/gcc/pic32mx/3.4.4/../../../../pic32mx/lib/size\libc.a(default-bootstrap-exception-handler.o)
                              C:/Program Files/Microchip/MPLAB C32 Suite/bin/../lib/gcc/pic32mx/3.4.4/../../../../pic32mx/lib/size/crt0.o (_bootstrap_exception_handler)
C:/Program Files/Microchip/MPLAB C32 Suite/bin/../lib/gcc/pic32mx/3.4.4/../../../../pic32mx/lib/size\libc.a(default-on-reset.o)
                              C:/Program Files/Microchip/MPLAB C32 Suite/bin/../lib/gcc/pic32mx/3.4.4/../../../../pic32mx/lib/size/crt0.o (_on_reset)
C:/Program Files/Microchip/MPLAB C32 Suite/bin/../lib/gcc/pic32mx/3.4.4/../../../../pic32mx/lib/size\libc.a(default-on-bootstrap.o)
                              C:/Program Files/Microchip/MPLAB C32 Suite/bin/../lib/gcc/pic32mx/3.4.4/../../../../pic32mx/lib/size/crt0.o (_on_bootstrap)
C:/Program Files/Microchip/MPLAB C32 Suite/bin/../lib/gcc/pic32mx/3.4.4/../../../../pic32mx/lib/size\libc.a(default-nmi-handler.o)
                              C:/Program Files/Microchip/MPLAB C32 Suite/bin/../lib/gcc/pic32mx/3.4.4/../../../../pic32mx/lib/size/crt0.o (_nmi_handler)
C:/Program Files/Microchip/MPLAB C32 Suite/bin/../lib/gcc/pic32mx/3.4.4/../../../../pic32mx/lib/size\libc.a(_mon_getc.o)
                              C:/Program Files/Microchip/MPLAB C32 Suite/bin/../lib/gcc/pic32mx/3.4.4/../../../../pic32mx/lib/size\libc.a(_iobfuncs.o) (_mon_getc)
C:/Program Files/Microchip/MPLAB C32 Suite/bin/../lib/gcc/pic32mx/3.4.4/../../../../pic32mx/lib/size\libc.a(_mon_write.o)
                              C:/Program Files/Microchip/MPLAB C32 Suite/bin/../lib/gcc/pic32mx/3.4.4/../../../../pic32mx/lib/size\libc.a(_iobfuncs.o) (_mon_write)
C:/Program Files/Microchip/MPLAB C32 Suite/bin/../lib/gcc/pic32mx/3.4.4/../../../../pic32mx/lib/size\libc.a(_exit.o)
                              C:/Program Files/Microchip/MPLAB C32 Suite/bin/../lib/gcc/pic32mx/3.4.4/../../../../pic32mx/lib/size\libc.a(exit.o) (_exit)
C:/Program Files/Microchip/MPLAB C32 Suite/bin/../lib/gcc/pic32mx/3.4.4/../../../../pic32mx/lib/size\libc.a(ctype.o)
                              C:/Program Files/Microchip/MPLAB C32 Suite/bin/../lib/gcc/pic32mx/3.4.4/../../../../pic32mx/lib/size\libc.a(strtol.o) (_ctype)
C:/Program Files/Microchip/MPLAB C32 Suite/bin/../lib/gcc/pic32mx/3.4.4/../../../../pic32mx/lib/size\libc.a(errno.o)
                              C:/Program Files/Microchip/MPLAB C32 Suite/bin/../lib/gcc/pic32mx/3.4.4/../../../../pic32mx/lib/size\libc.a(strtol.o) (errno)
C:/Program Files/Microchip/MPLAB C32 Suite/bin/../lib/gcc/pic32mx/3.4.4/../../../../pic32mx/lib/size\libc.a(_mon_putc.o)
                              C:/Program Files/Microchip/MPLAB C32 Suite/bin/../lib/gcc/pic32mx/3.4.4/../../../../pic32mx/lib/size\libc.a(_mon_write.o) (_mon_putc)
C:/Program Files/Microchip/MPLAB C32 Suite/bin/../lib/gcc/pic32mx/3.4.4/../../../../pic32mx/lib/size\libmchp_peripheral.a(int_disable_interrupts_lib.o)
                              Objects - TCPIP Demo App-C32\MainDemo.o (INTDisableInterrupts)
C:/Program Files/Microchip/MPLAB C32 Suite/bin/../lib/gcc/pic32mx/3.4.4/../../../../pic32mx/lib/size\libmchp_peripheral.a(int_enable_mv_int_lib.o)
                              Objects - TCPIP Demo App-C32\MainDemo.o (INTEnableSystemMultiVectoredInt)
C:/Program Files/Microchip/MPLAB C32 Suite/bin/../lib/gcc/pic32mx/3.4.4/../../../../pic32mx/lib/size\libmchp_peripheral.a(int_restore_interrupts_lib.o)
                              Objects - TCPIP Demo App-C32\MainDemo.o (INTRestoreInterrupts)
C:/Program Files/Microchip/MPLAB C32 Suite/bin/../lib/gcc/pic32mx/3.4.4/../../../../pic32mx/lib/size\libmchp_peripheral.a(puts_uartx_lib.o)
                              Objects - TCPIP Demo App-C32\MainDemo.o (putsUART2)
C:/Program Files/Microchip/MPLAB C32 Suite/bin/../lib/gcc/pic32mx/3.4.4/../../../../pic32mx/lib/size\libmchp_peripheral.a(soft_reset_lib.o)
                              Objects - TCPIP Demo App-C32\MainDemo.o (SoftReset)
C:/Program Files/Microchip/MPLAB C32 Suite/bin/../lib/gcc/pic32mx/3.4.4/../../../../pic32mx/lib/size\libmchp_peripheral.a(pcache.o)
                              Objects - TCPIP Demo App-C32\MainDemo.o (CheKseg0CacheOn)
C:/Program Files/Microchip/MPLAB C32 Suite/bin/../lib/gcc/pic32mx/3.4.4/../../../../pic32mx/lib/size\libmchp_peripheral.a(int_enable_interrupts_lib.o)
                              C:/Program Files/Microchip/MPLAB C32 Suite/bin/../lib/gcc/pic32mx/3.4.4/../../../../pic32mx/lib/size\libmchp_peripheral.a(int_enable_mv_int_lib.o) (INTEnableInterrupts)

Allocating common symbols
Common symbol       size              file

UDPTxCount          0x2               ..\Microchip\TCPIP Stack\Objects - TCPIP Demo App-C32\UDP.o
LCDText             0x21              ..\Microchip\TCPIP Stack\Objects - TCPIP Demo App-C32\LCDBlocking.o
curHTTP             0x8c              ..\Microchip\TCPIP Stack\Objects - TCPIP Demo App-C32\HTTP2.o
snmpReqVarErrStatus
                    0x8               ..\Microchip\TCPIP Stack\Objects - TCPIP Demo App-C32\SNMP.o
activeUDPSocket     0x1               ..\Microchip\TCPIP Stack\Objects - TCPIP Demo App-C32\UDP.o
curHTTPID           0x1               ..\Microchip\TCPIP Stack\Objects - TCPIP Demo App-C32\HTTP2.o
remoteNode          0xa               ..\Microchip\TCPIP Stack\Objects - TCPIP Demo App-C32\StackTsk.o
DDNSClient          0x20              ..\Microchip\TCPIP Stack\Objects - TCPIP Demo App-C32\DynDNS.o
SMTPClient          0x2c              ..\Microchip\TCPIP Stack\Objects - TCPIP Demo App-C32\SMTP.o
lastBlock           0x40              ..\Microchip\TCPIP Stack\Objects - TCPIP Demo App-C32\Hashes.o
AppConfig           0x69              Objects - TCPIP Demo App-C32\MainDemo.o
UDPRxCount          0x2               ..\Microchip\TCPIP Stack\Objects - TCPIP Demo App-C32\UDP.o
lastRead            0x4               ..\Microchip\TCPIP Stack\Objects - TCPIP Demo App-C32\MPFS2.o
UDPSocketInfo       0x8c              ..\Microchip\TCPIP Stack\Objects - TCPIP Demo App-C32\UDP.o
httpStubs           0x10              ..\Microchip\TCPIP Stack\Objects - TCPIP Demo App-C32\HTTP2.o
AN0String           0x8               Objects - TCPIP Demo App-C32\MainDemo.o

Memory Configuration

Name             Origin             Length             Attributes
kseg0_program_mem 0x9d000000         0x00080000         xr
kseg0_boot_mem   0x9fc00490         0x00000970
exception_mem    0x9fc01000         0x00001000
kseg1_boot_mem   0xbfc00000         0x00000490
debug_exec_mem   0xbfc02000         0x00000ff0
config3          0xbfc02ff0         0x00000004
config2          0xbfc02ff4         0x00000004
config1          0xbfc02ff8         0x00000004
config0          0xbfc02ffc         0x00000004
kseg1_data_mem   0xa0000000         0x00008000         w !x
sfrs             0xbf800000         0x00100000
*default*        0x00000000         0xffffffff

Linker script and memory map

LOAD C:/Program Files/Microchip/MPLAB C32 Suite/bin/../lib/gcc/pic32mx/3.4.4/../../../../pic32mx/lib/size/crt0.o
LOAD Objects - TCPIP Demo App-C32\MainDemo.o
LOAD Objects - TCPIP Demo App-C32\CustomHTTPApp.o
LOAD ..\Microchip\TCPIP Stack\Objects - TCPIP Demo App-C32\UDPPerformanceTest.o
LOAD ..\Microchip\TCPIP Stack\Objects - TCPIP Demo App-C32\Announce.o
LOAD ..\Microchip\TCPIP Stack\Objects - TCPIP Demo App-C32\ARP.o
LOAD ..\Microchip\TCPIP Stack\Objects - TCPIP Demo App-C32\Delay.o
LOAD ..\Microchip\TCPIP Stack\Objects - TCPIP Demo App-C32\DHCP.o
LOAD ..\Microchip\TCPIP Stack\Objects - TCPIP Demo App-C32\DHCPs.o
LOAD ..\Microchip\TCPIP Stack\Objects - TCPIP Demo App-C32\DNS.o
LOAD ..\Microchip\TCPIP Stack\Objects - TCPIP Demo App-C32\DynDNS.o
LOAD ..\Microchip\TCPIP Stack\Objects - TCPIP Demo App-C32\ENC28J60.o
LOAD ..\Microchip\TCPIP Stack\Objects - TCPIP Demo App-C32\FTP.o
LOAD ..\Microchip\TCPIP Stack\Objects - TCPIP Demo App-C32\Hashes.o
LOAD ..\Microchip\TCPIP Stack\Objects - TCPIP Demo App-C32\Helpers.o
LOAD ..\Microchip\TCPIP Stack\Objects - TCPIP Demo App-C32\HTTP2.o
LOAD ..\Microchip\TCPIP Stack\Objects - TCPIP Demo App-C32\HTTP.o
LOAD ..\Microchip\TCPIP Stack\Objects - TCPIP Demo App-C32\ICMP.o
LOAD ..\Microchip\TCPIP Stack\Objects - TCPIP Demo App-C32\IP.o
LOAD ..\Microchip\TCPIP Stack\Objects - TCPIP Demo App-C32\LCDBlocking.o
LOAD ..\Microchip\TCPIP Stack\Objects - TCPIP Demo App-C32\MPFS2.o
LOAD ..\Microchip\TCPIP Stack\Objects - TCPIP Demo App-C32\MPFS.o
LOAD ..\Microchip\TCPIP Stack\Objects - TCPIP Demo App-C32\NBNS.o
LOAD ..\Microchip\TCPIP Stack\Objects - TCPIP Demo App-C32\Reboot.o
LOAD ..\Microchip\TCPIP Stack\Objects - TCPIP Demo App-C32\SMTP.o
LOAD ..\Microchip\TCPIP Stack\Objects - TCPIP Demo App-C32\SNMP.o
LOAD ..\Microchip\TCPIP Stack\Objects - TCPIP Demo App-C32\SNTP.o
LOAD ..\Microchip\TCPIP Stack\Objects - TCPIP Demo App-C32\SPIEEPROM.o
LOAD ..\Microchip\TCPIP Stack\Objects - TCPIP Demo App-C32\SPIFlash.o
LOAD ..\Microchip\TCPIP Stack\Objects - TCPIP Demo App-C32\SPIRAM.o
LOAD ..\Microchip\TCPIP Stack\Objects - TCPIP Demo App-C32\StackTsk.o
LOAD ..\Microchip\TCPIP Stack\Objects - TCPIP Demo App-C32\TCP.o
LOAD ..\Microchip\TCPIP Stack\Objects - TCPIP Demo App-C32\TCPPerformanceTest.o
LOAD ..\Microchip\TCPIP Stack\Objects - TCPIP Demo App-C32\Telnet.o
LOAD ..\Microchip\TCPIP Stack\Objects - TCPIP Demo App-C32\TFTPc.o
LOAD ..\Microchip\TCPIP Stack\Objects - TCPIP Demo App-C32\Tick.o
LOAD ..\Microchip\TCPIP Stack\Objects - TCPIP Demo App-C32\UART2TCPBridge.o
LOAD ..\Microchip\TCPIP Stack\Objects - TCPIP Demo App-C32\UART.o
LOAD ..\Microchip\TCPIP Stack\Objects - TCPIP Demo App-C32\UDP.o
LOAD Objects - TCPIP Demo App-C32\CustomSNMPApp.o
LOAD Objects - TCPIP Demo App-C32\UARTConfig.o
LOAD Objects - TCPIP Demo App-C32\GenericTCPClient.o
LOAD Objects - TCPIP Demo App-C32\GenericTCPServer.o
LOAD Objects - TCPIP Demo App-C32\LegacyHTTPApp.o
LOAD Objects - TCPIP Demo App-C32\PingDemo.o
LOAD Objects - TCPIP Demo App-C32\SMTPDemo.o
LOAD ..\Microchip\TCPIP Stack\Objects - TCPIP Demo App-C32\BerkeleyAPI.o
LOAD Objects - TCPIP Demo App-C32\BerkeleyUDPClientDemo.o
LOAD Objects - TCPIP Demo App-C32\BerkeleyTCPClientDemo.o
LOAD Objects - TCPIP Demo App-C32\BerkeleyTCPServerDemo.o
LOAD ..\Microchip\TCPIP Stack\Objects - TCPIP Demo App-C32\ENCX24J600.o
LOAD Objects - TCPIP Demo App-C32\MPFSImg2.o
LOAD ..\Microchip\TCPIP Stack\Objects - TCPIP Demo App-C32\Random.o
LOAD ..\Microchip\TCPIP Stack\Objects - TCPIP Demo App-C32\RSA.o
LOAD ..\Microchip\TCPIP Stack\Objects - TCPIP Demo App-C32\SSL.o
LOAD ..\Microchip\TCPIP Stack\Objects - TCPIP Demo App-C32\ARCFOUR.o
LOAD ..\Microchip\TCPIP Stack\Objects - TCPIP Demo App-C32\BigInt.o
LOAD ..\Microchip\TCPIP Stack\Objects - TCPIP Demo App-C32\BigInt_helper_C32.o
LOAD Objects - TCPIP Demo App-C32\CustomSSLCert.o
                0x00000001                __MPLAB_BUILD = 0x1
LOAD C:/Program Files/Microchip/MPLAB C32 Suite/bin/../lib/gcc/pic32mx/3.4.4/size\libgcc.a
START GROUP
LOAD C:/Program Files/Microchip/MPLAB C32 Suite/bin/../lib/gcc/pic32mx/3.4.4/../../../../pic32mx/lib/size\libc.a
LOAD C:/Program Files/Microchip/MPLAB C32 Suite/bin/../lib/gcc/pic32mx/3.4.4/../../../../pic32mx/lib/size\libm.a
LOAD C:/Program Files/Microchip/MPLAB C32 Suite/bin/../lib/gcc/pic32mx/3.4.4/../../../../pic32mx/lib/size\libe.a
LOAD C:/Program Files/Microchip/MPLAB C32 Suite/bin/../lib/gcc/pic32mx/3.4.4/../../../../pic32mx/lib/size\libdsp.a
LOAD C:/Program Files/Microchip/MPLAB C32 Suite/bin/../lib/gcc/pic32mx/3.4.4/../../../../pic32mx/lib/size\libmchp_peripheral.a
LOAD C:/Program Files/Microchip/MPLAB C32 Suite/bin/../lib/gcc/pic32mx/3.4.4/../../../../pic32mx/lib/size\libmchp_peripheral_32MX360F512L.a
END GROUP
LOAD C:/Program Files/Microchip/MPLAB C32 Suite/bin/../lib/gcc/pic32mx/3.4.4/size\libgcc.a
                0x00000400                PROVIDE (_min_stack_size, 0x400)
                0x00000000                PROVIDE (_min_heap_size, 0x0)
LOAD C:/Program Files/Microchip/MPLAB C32 Suite/bin/../lib/gcc/pic32mx/3.4.4/../../../../pic32mx/lib/./proc/32MX360F512L\processor.o
                0x00000001                PROVIDE (_vector_spacing, 0x1)
                0x9fc01000                _ebase_address = 0x9fc01000
                0xbfc00000                _RESET_ADDR = 0xbfc00000
                0xbfc00380                _BEV_EXCPT_ADDR = 0xbfc00380
                0xbfc00480                _DBG_EXCPT_ADDR = 0xbfc00480
                0xbfc02000                _DBG_CODE_ADDR = 0xbfc02000
                0x9fc01180                _GEN_EXCPT_ADDR = (_ebase_address + 0x180)

.config_BFC02FF0
 *(.config_BFC02FF0)

.config_BFC02FF4
                0xbfc02ff4        0x4
 *(.config_BFC02FF4)
 .config_BFC02FF4
                0xbfc02ff4        0x4 Objects - TCPIP Demo App-C32\MainDemo.o

.config_BFC02FF8
                0xbfc02ff8        0x4
 *(.config_BFC02FF8)
 .config_BFC02FF8
                0xbfc02ff8        0x4 Objects - TCPIP Demo App-C32\MainDemo.o

.config_BFC02FFC
                0xbfc02ffc        0x4
 *(.config_BFC02FFC)
 .config_BFC02FFC
                0xbfc02ffc        0x4 Objects - TCPIP Demo App-C32\MainDemo.o

.reset          0xbfc00000       0x10
 *(.reset)
 .reset         0xbfc00000       0x10 C:/Program Files/Microchip/MPLAB C32 Suite/bin/../lib/gcc/pic32mx/3.4.4/../../../../pic32mx/lib/size/crt0.o
                0xbfc00000                _reset

.bev_excpt      0xbfc00380       0x10
 *(.bev_handler)
 .bev_handler   0xbfc00380       0x10 C:/Program Files/Microchip/MPLAB C32 Suite/bin/../lib/gcc/pic32mx/3.4.4/../../../../pic32mx/lib/size/crt0.o

.dbg_excpt      0xbfc00480        0x0
                0xbfc00480                . = (. + DEFINED (_DEBUGGER)?0x8:0x0)

.dbg_code       0xbfc02000        0x0
                0xbfc02000                . = (. + DEFINED (_DEBUGGER)?0xff0:0x0)

.app_excpt      0x9fc01180       0x10
 *(.gen_handler)
 .gen_handler   0x9fc01180       0x10 C:/Program Files/Microchip/MPLAB C32 Suite/bin/../lib/gcc/pic32mx/3.4.4/../../../../pic32mx/lib/size/crt0.o

.vector_0       0x9fc01200        0x0
 *(.vector_0)
                0x00000001                ASSERT (((_vector_spacing == 0x0) || (SIZEOF (.vector_0) <= (_vector_spacing << 0x5))), function at exception vector 0 too large)

.vector_1       0x9fc01220        0x0
 *(.vector_1)
                0x00000001                ASSERT (((_vector_spacing == 0x0) || (SIZEOF (.vector_1) <= (_vector_spacing << 0x5))), function at exception vector 1 too large)

.vector_2       0x9fc01240        0x0
 *(.vector_2)
                0x00000001                ASSERT (((_vector_spacing == 0x0) || (SIZEOF (.vector_2) <= (_vector_spacing << 0x5))), function at exception vector 2 too large)

.vector_3       0x9fc01260        0x0
 *(.vector_3)
                0x00000001                ASSERT (((_vector_spacing == 0x0) || (SIZEOF (.vector_3) <= (_vector_spacing << 0x5))), function at exception vector 3 too large)

.vector_4       0x9fc01280        0x8
 *(.vector_4)
 .vector_4      0x9fc01280        0x8 ..\Microchip\TCPIP Stack\Objects - TCPIP Demo App-C32\Tick.o
                0x00000001                ASSERT (((_vector_spacing == 0x0) || (SIZEOF (.vector_4) <= (_vector_spacing << 0x5))), function at exception vector 4 too large)

.vector_5       0x9fc012a0        0x0
 *(.vector_5)
                0x00000001                ASSERT (((_vector_spacing == 0x0) || (SIZEOF (.vector_5) <= (_vector_spacing << 0x5))), function at exception vector 5 too large)

.vector_6       0x9fc012c0        0x0
 *(.vector_6)
                0x00000001                ASSERT (((_vector_spacing == 0x0) || (SIZEOF (.vector_6) <= (_vector_spacing << 0x5))), function at exception vector 6 too large)

.vector_7       0x9fc012e0        0x0
 *(.vector_7)
                0x00000001                ASSERT (((_vector_spacing == 0x0) || (SIZEOF (.vector_7) <= (_vector_spacing << 0x5))), function at exception vector 7 too large)

.vector_8       0x9fc01300        0x0
 *(.vector_8)
                0x00000001                ASSERT (((_vector_spacing == 0x0) || (SIZEOF (.vector_8) <= (_vector_spacing << 0x5))), function at exception vector 8 too large)

.vector_9       0x9fc01320        0x0
 *(.vector_9)
                0x00000001                ASSERT (((_vector_spacing == 0x0) || (SIZEOF (.vector_9) <= (_vector_spacing << 0x5))), function at exception vector 9 too large)

.vector_10      0x9fc01340        0x0
 *(.vector_10)
                0x00000001                ASSERT (((_vector_spacing == 0x0) || (SIZEOF (.vector_10) <= (_vector_spacing << 0x5))), function at exception vector 10 too large)

.vector_11      0x9fc01360        0x0
 *(.vector_11)
                0x00000001                ASSERT (((_vector_spacing == 0x0) || (SIZEOF (.vector_11) <= (_vector_spacing << 0x5))), function at exception vector 11 too large)

.vector_12      0x9fc01380        0x0
 *(.vector_12)
                0x00000001                ASSERT (((_vector_spacing == 0x0) || (SIZEOF (.vector_12) <= (_vector_spacing << 0x5))), function at exception vector 12 too large)

.vector_13      0x9fc013a0        0x0
 *(.vector_13)
                0x00000001                ASSERT (((_vector_spacing == 0x0) || (SIZEOF (.vector_13) <= (_vector_spacing << 0x5))), function at exception vector 13 too large)

.vector_14      0x9fc013c0        0x0
 *(.vector_14)
                0x00000001                ASSERT (((_vector_spacing == 0x0) || (SIZEOF (.vector_14) <= (_vector_spacing << 0x5))), function at exception vector 14 too large)

.vector_15      0x9fc013e0        0x0
 *(.vector_15)
                0x00000001                ASSERT (((_vector_spacing == 0x0) || (SIZEOF (.vector_15) <= (_vector_spacing << 0x5))), function at exception vector 15 too large)

.vector_16      0x9fc01400        0x0
 *(.vector_16)
                0x00000001                ASSERT (((_vector_spacing == 0x0) || (SIZEOF (.vector_16) <= (_vector_spacing << 0x5))), function at exception vector 16 too large)

.vector_17      0x9fc01420        0x0
 *(.vector_17)
                0x00000001                ASSERT (((_vector_spacing == 0x0) || (SIZEOF (.vector_17) <= (_vector_spacing << 0x5))), function at exception vector 17 too large)

.vector_18      0x9fc01440        0x0
 *(.vector_18)
                0x00000001                ASSERT (((_vector_spacing == 0x0) || (SIZEOF (.vector_18) <= (_vector_spacing << 0x5))), function at exception vector 18 too large)

.vector_19      0x9fc01460        0x0
 *(.vector_19)
                0x00000001                ASSERT (((_vector_spacing == 0x0) || (SIZEOF (.vector_19) <= (_vector_spacing << 0x5))), function at exception vector 19 too large)

.vector_20      0x9fc01480        0x0
 *(.vector_20)
                0x00000001                ASSERT (((_vector_spacing == 0x0) || (SIZEOF (.vector_20) <= (_vector_spacing << 0x5))), function at exception vector 20 too large)

.vector_21      0x9fc014a0        0x0
 *(.vector_21)
                0x00000001                ASSERT (((_vector_spacing == 0x0) || (SIZEOF (.vector_21) <= (_vector_spacing << 0x5))), function at exception vector 21 too large)

.vector_22      0x9fc014c0        0x0
 *(.vector_22)
                0x00000001                ASSERT (((_vector_spacing == 0x0) || (SIZEOF (.vector_22) <= (_vector_spacing << 0x5))), function at exception vector 22 too large)

.vector_23      0x9fc014e0        0x0
 *(.vector_23)
                0x00000001                ASSERT (((_vector_spacing == 0x0) || (SIZEOF (.vector_23) <= (_vector_spacing << 0x5))), function at exception vector 23 too large)

.vector_24      0x9fc01500        0x0
 *(.vector_24)
                0x00000001                ASSERT (((_vector_spacing == 0x0) || (SIZEOF (.vector_24) <= (_vector_spacing << 0x5))), function at exception vector 24 too large)

.vector_25      0x9fc01520        0x0
 *(.vector_25)
                0x00000001                ASSERT (((_vector_spacing == 0x0) || (SIZEOF (.vector_25) <= (_vector_spacing << 0x5))), function at exception vector 25 too large)

.vector_26      0x9fc01540        0x0
 *(.vector_26)
                0x00000001                ASSERT (((_vector_spacing == 0x0) || (SIZEOF (.vector_26) <= (_vector_spacing << 0x5))), function at exception vector 26 too large)

.vector_27      0x9fc01560        0x0
 *(.vector_27)
                0x00000001                ASSERT (((_vector_spacing == 0x0) || (SIZEOF (.vector_27) <= (_vector_spacing << 0x5))), function at exception vector 27 too large)

.vector_28      0x9fc01580        0x0
 *(.vector_28)
                0x00000001                ASSERT (((_vector_spacing == 0x0) || (SIZEOF (.vector_28) <= (_vector_spacing << 0x5))), function at exception vector 28 too large)

.vector_29      0x9fc015a0        0x0
 *(.vector_29)
                0x00000001                ASSERT (((_vector_spacing == 0x0) || (SIZEOF (.vector_29) <= (_vector_spacing << 0x5))), function at exception vector 29 too large)

.vector_30      0x9fc015c0        0x0
 *(.vector_30)
                0x00000001                ASSERT (((_vector_spacing == 0x0) || (SIZEOF (.vector_30) <= (_vector_spacing << 0x5))), function at exception vector 30 too large)

.vector_31      0x9fc015e0        0x0
 *(.vector_31)
                0x00000001                ASSERT (((_vector_spacing == 0x0) || (SIZEOF (.vector_31) <= (_vector_spacing << 0x5))), function at exception vector 31 too large)

.vector_32      0x9fc01600        0x8
 *(.vector_32)
 .vector_32     0x9fc01600        0x8 ..\Microchip\TCPIP Stack\Objects - TCPIP Demo App-C32\UART2TCPBridge.o
                0x00000001                ASSERT (((_vector_spacing == 0x0) || (SIZEOF (.vector_32) <= (_vector_spacing << 0x5))), function at exception vector 32 too large)

.vector_33      0x9fc01620        0x0
 *(.vector_33)
                0x00000001                ASSERT (((_vector_spacing == 0x0) || (SIZEOF (.vector_33) <= (_vector_spacing << 0x5))), function at exception vector 33 too large)

.vector_34      0x9fc01640        0x0
 *(.vector_34)
                0x00000001                ASSERT (((_vector_spacing == 0x0) || (SIZEOF (.vector_34) <= (_vector_spacing << 0x5))), function at exception vector 34 too large)

.vector_35      0x9fc01660        0x0
 *(.vector_35)
                0x00000001                ASSERT (((_vector_spacing == 0x0) || (SIZEOF (.vector_35) <= (_vector_spacing << 0x5))), function at exception vector 35 too large)

.vector_36      0x9fc01680        0x0
 *(.vector_36)
                0x00000001                ASSERT (((_vector_spacing == 0x0) || (SIZEOF (.vector_36) <= (_vector_spacing << 0x5))), function at exception vector 36 too large)

.vector_37      0x9fc016a0        0x0
 *(.vector_37)
                0x00000001                ASSERT (((_vector_spacing == 0x0) || (SIZEOF (.vector_37) <= (_vector_spacing << 0x5))), function at exception vector 37 too large)

.vector_38      0x9fc016c0        0x0
 *(.vector_38)
                0x00000001                ASSERT (((_vector_spacing == 0x0) || (SIZEOF (.vector_38) <= (_vector_spacing << 0x5))), function at exception vector 38 too large)

.vector_39      0x9fc016e0        0x0
 *(.vector_39)
                0x00000001                ASSERT (((_vector_spacing == 0x0) || (SIZEOF (.vector_39) <= (_vector_spacing << 0x5))), function at exception vector 39 too large)

.vector_40      0x9fc01700        0x0
 *(.vector_40)
                0x00000001                ASSERT (((_vector_spacing == 0x0) || (SIZEOF (.vector_40) <= (_vector_spacing << 0x5))), function at exception vector 40 too large)

.vector_41      0x9fc01720        0x0
 *(.vector_41)
                0x00000001                ASSERT (((_vector_spacing == 0x0) || (SIZEOF (.vector_41) <= (_vector_spacing << 0x5))), function at exception vector 41 too large)

.vector_42      0x9fc01740        0x0
 *(.vector_42)
                0x00000001                ASSERT (((_vector_spacing == 0x0) || (SIZEOF (.vector_42) <= (_vector_spacing << 0x5))), function at exception vector 42 too large)

.vector_43      0x9fc01760        0x0
 *(.vector_43)
                0x00000001                ASSERT (((_vector_spacing == 0x0) || (SIZEOF (.vector_43) <= (_vector_spacing << 0x5))), function at exception vector 43 too large)

.vector_44      0x9fc01780        0x0
 *(.vector_44)
                0x00000001                ASSERT (((_vector_spacing == 0x0) || (SIZEOF (.vector_44) <= (_vector_spacing << 0x5))), function at exception vector 44 too large)

.vector_45      0x9fc017a0        0x0
 *(.vector_45)
                0x00000001                ASSERT (((_vector_spacing == 0x0) || (SIZEOF (.vector_45) <= (_vector_spacing << 0x5))), function at exception vector 45 too large)

.vector_46      0x9fc017c0        0x0
 *(.vector_46)
                0x00000001                ASSERT (((_vector_spacing == 0x0) || (SIZEOF (.vector_46) <= (_vector_spacing << 0x5))), function at exception vector 46 too large)

.vector_47      0x9fc017e0        0x0
 *(.vector_47)
                0x00000001                ASSERT (((_vector_spacing == 0x0) || (SIZEOF (.vector_47) <= (_vector_spacing << 0x5))), function at exception vector 47 too large)

.vector_48      0x9fc01800        0x0
 *(.vector_48)
                0x00000001                ASSERT (((_vector_spacing == 0x0) || (SIZEOF (.vector_48) <= (_vector_spacing << 0x5))), function at exception vector 48 too large)

.vector_49      0x9fc01820        0x0
 *(.vector_49)
                0x00000001                ASSERT (((_vector_spacing == 0x0) || (SIZEOF (.vector_49) <= (_vector_spacing << 0x5))), function at exception vector 49 too large)

.vector_50      0x9fc01840        0x0
 *(.vector_50)
                0x00000001                ASSERT (((_vector_spacing == 0x0) || (SIZEOF (.vector_50) <= (_vector_spacing << 0x5))), function at exception vector 50 too large)

.vector_51      0x9fc01860        0x0
 *(.vector_51)
                0x00000001                ASSERT (((_vector_spacing == 0x0) || (SIZEOF (.vector_51) <= (_vector_spacing << 0x5))), function at exception vector 51 too large)

.vector_52      0x9fc01880        0x0
 *(.vector_52)
                0x00000001                ASSERT (((_vector_spacing == 0x0) || (SIZEOF (.vector_52) <= (_vector_spacing << 0x5))), function at exception vector 52 too large)

.vector_53      0x9fc018a0        0x0
 *(.vector_53)
                0x00000001                ASSERT (((_vector_spacing == 0x0) || (SIZEOF (.vector_53) <= (_vector_spacing << 0x5))), function at exception vector 53 too large)

.vector_54      0x9fc018c0        0x0
 *(.vector_54)
                0x00000001                ASSERT (((_vector_spacing == 0x0) || (SIZEOF (.vector_54) <= (_vector_spacing << 0x5))), function at exception vector 54 too large)

.vector_55      0x9fc018e0        0x0
 *(.vector_55)
                0x00000001                ASSERT (((_vector_spacing == 0x0) || (SIZEOF (.vector_55) <= (_vector_spacing << 0x5))), function at exception vector 55 too large)

.vector_56      0x9fc01900        0x0
 *(.vector_56)
                0x00000001                ASSERT (((_vector_spacing == 0x0) || (SIZEOF (.vector_56) <= (_vector_spacing << 0x5))), function at exception vector 56 too large)

.vector_57      0x9fc01920        0x0
 *(.vector_57)
                0x00000001                ASSERT (((_vector_spacing == 0x0) || (SIZEOF (.vector_57) <= (_vector_spacing << 0x5))), function at exception vector 57 too large)

.vector_58      0x9fc01940        0x0
 *(.vector_58)
                0x00000001                ASSERT (((_vector_spacing == 0x0) || (SIZEOF (.vector_58) <= (_vector_spacing << 0x5))), function at exception vector 58 too large)

.vector_59      0x9fc01960        0x0
 *(.vector_59)
                0x00000001                ASSERT (((_vector_spacing == 0x0) || (SIZEOF (.vector_59) <= (_vector_spacing << 0x5))), function at exception vector 59 too large)

.vector_60      0x9fc01980        0x0
 *(.vector_60)
                0x00000001                ASSERT (((_vector_spacing == 0x0) || (SIZEOF (.vector_60) <= (_vector_spacing << 0x5))), function at exception vector 60 too large)

.vector_61      0x9fc019a0        0x0
 *(.vector_61)
                0x00000001                ASSERT (((_vector_spacing == 0x0) || (SIZEOF (.vector_61) <= (_vector_spacing << 0x5))), function at exception vector 61 too large)

.vector_62      0x9fc019c0        0x0
 *(.vector_62)
                0x00000001                ASSERT (((_vector_spacing == 0x0) || (SIZEOF (.vector_62) <= (_vector_spacing << 0x5))), function at exception vector 62 too large)

.vector_63      0x9fc019e0        0x0
 *(.vector_63)
                0x00000001                ASSERT (((_vector_spacing == 0x0) || (SIZEOF (.vector_63) <= (_vector_spacing << 0x5))), function at exception vector 63 too large)

.startup        0x9fc00490      0x1e0
 *(.startup)
 .startup       0x9fc00490      0x1e0 C:/Program Files/Microchip/MPLAB C32 Suite/bin/../lib/gcc/pic32mx/3.4.4/../../../../pic32mx/lib/size/crt0.o

.text           0x9d000000    0x2d274
                0x9d000000                _text_begin = .
 *(.text .stub .text.* .gnu.linkonce.t.*)
 .text          0x9d000000       0x18 C:/Program Files/Microchip/MPLAB C32 Suite/bin/../lib/gcc/pic32mx/3.4.4/../../../../pic32mx/lib/size/crt0.o
 .text          0x9d000018      0xf0c Objects - TCPIP Demo App-C32\MainDemo.o
                0x9d000ed0                SaveAppConfig
                0x9d000044                main
                0x9d0002f0                DisplayIPValue
                0x9d000018                _general_exception_handler
 .text          0x9d000f24     0x3ea8 Objects - TCPIP Demo App-C32\CustomHTTPApp.o
                0x9d003a2c                HTTPPrint_lcdtext
                0x9d004230                HTTPPrint_config_dns2
                0x9d004bf4                HTTPPrint_smtps_en
                0x9d004844                HTTPPrint_ddns_service
                0x9d004520                HTTPPrint_rebootaddr
                0x9d00404c                HTTPPrint_config_hostname
                0x9d0039bc                HTTPPrint_pot
                0x9d003f7c                HTTPPrintIP
                0x9d000f24                HTTPNeedsAuth
                0x9d004468                HTTPPrint_write_comm
                0x9d0041a0                HTTPPrint_config_subnet
                0x9d004574                HTTPPrint_ddns_user
                0x9d0043e0                HTTPPrint_read_comm
                0x9d004c48                HTTPPrint_snmp_en
                0x9d003c38                HTTPPrint_hellomsg
                0x9d004c9c                HTTPPrint_status_ok
                0x9d00350c                HTTPPrint_version
                0x9d003cdc                HTTPPrint_cookiename
                0x9d0041e8                HTTPPrint_config_dns1
                0x9d004158                HTTPPrint_config_gw
                0x9d004a0c                HTTPPrint_ddns_status_msg
                0x9d001440                HTTPExecutePost
                0x9d003d88                HTTPPrint_uploadedmd5
                0x9d0036b0                HTTPPrint_led
                0x9d00382c                HTTPPrint_ledSelected
                0x9d004900                HTTPPrint_ddns_status
                0x9d000fe4                HTTPCheckAuth
                0x9d0044f0                HTTPPrint_reboot
                0x9d004664                HTTPPrint_ddns_pass
                0x9d0010d8                HTTPExecuteGet
                0x9d0040a0                HTTPPrint_config_dhcpchecked
                0x9d004d34                HTTPPrint_status_fail
                0x9d003560                HTTPPrint_btn
                0x9d004110                HTTPPrint_config_ip
                0x9d004754                HTTPPrint_ddns_host
                0x9d004278                HTTPPrint_config_mac
                0x9d003464                HTTPPrint_builddate
 .text          0x9d004dcc      0x3a4 ..\Microchip\TCPIP Stack\Objects - TCPIP Demo App-C32\Announce.o
                0x9d004dcc                AnnounceIP
                0x9d004f2c                DiscoveryTask
 .text          0x9d005170      0x5ec ..\Microchip\TCPIP Stack\Objects - TCPIP Demo App-C32\ARP.o
                0x9d0055d4                ARPIsResolved
                0x9d005304                ARPProcess
                0x9d005274                ARPInit
                0x9d0054f4                ARPResolve
 .text          0x9d00575c       0xe8 ..\Microchip\TCPIP Stack\Objects - TCPIP Demo App-C32\Delay.o
                0x9d00575c                DelayMs
                0x9d0057e0                Delay10us
 .text          0x9d005844     0x11d4 ..\Microchip\TCPIP Stack\Objects - TCPIP Demo App-C32\DHCP.o
                0x9d005844                DHCPReset
                0x9d00597c                DHCPTask
                0x9d0058b4                DHCPDisable
                0x9d005920                DHCPEnable
 .text          0x9d006a18      0xae0 ..\Microchip\TCPIP Stack\Objects - TCPIP Demo App-C32\DHCPs.o
                0x9d006a18                DHCPServerTask
 .text          0x9d0074f8      0xe9c ..\Microchip\TCPIP Stack\Objects - TCPIP Demo App-C32\DNS.o
                0x9d007550                DNSEndUsage
                0x9d0075c4                DNSResolve
                0x9d007658                DNSIsResolved
                0x9d0074f8                DNSBeginUsage
 .text          0x9d008394     0x1788 ..\Microchip\TCPIP Stack\Objects - TCPIP Demo App-C32\DynDNS.o
                0x9d009ac8                DDNSGetLastIP
                0x9d009a48                DDNSSetService
                0x9d008434                DDNSTask
                0x9d008394                DDNSInit
                0x9d009af8                DDNSGetLastStatus
                0x9d009a04                DDNSForceUpdate
 .text          0x9d009b1c     0x24f8 ..\Microchip\TCPIP Stack\Objects - TCPIP Demo App-C32\ENC28J60.o
                0x9d009eb0                MACIsTxReady
                0x9d00ab70                MACMemCopyAsync
                0x9d00b3f8                MACPutArray
                0x9d00a720                MACSetReadPtrInRx
                0x9d009b1c                MACInit
                0x9d00a9d8                CalcIPBufferChecksum
                0x9d00a124                MACGetHeader
                0x9d009efc                MACDiscardRx
                0x9d00a8d0                MACCalcRxChecksum
                0x9d00bd28                WritePHYReg
                0x9d00bf58                SetCLKOUT
                0x9d00be40                MACPowerDown
                0x9d00a3f8                MACFlush
                0x9d00a7a8                MACSetWritePtr
                0x9d00afb0                MACIsMemCopyDone
                0x9d00bee4                MACPowerUp
                0x9d00b33c                MACPut
                0x9d009e70                MACIsLinked
                0x9d00b0b0                MACGetArray
                0x9d00affc                MACGet
                0x9d00bfb4                GetCLKOUT
                0x9d00a83c                MACSetReadPtr
                0x9d009f9c                MACGetFreeRxSize
                0x9d00b964                ReadPHYReg
                0x9d00a30c                MACPutHeader
 .text          0x9d00c014      0x76c ..\Microchip\TCPIP Stack\Objects - TCPIP Demo App-C32\Hashes.o
                0x9d00c4a4                MD5Calculate
                0x9d00c014                HashAddData
                0x9d00c074                MD5Initialize
                0x9d00c0e8                MD5AddData
 .text          0x9d00c780     0x13b4 ..\Microchip\TCPIP Stack\Objects - TCPIP Demo App-C32\Helpers.o
                0x9d00d2bc                uitoa
                0x9d00d884                swapl
                0x9d00d5d8                btohexa_high
                0x9d00d838                swaps
                0x9d00c9c8                StringToIPAddress
                0x9d00da7c                FormatNetBIOSName
                0x9d00d648                btohexa_low
                0x9d00d90c                CalcIPChecksum
                0x9d00d504                hexatob
                0x9d00d6b8                stricmppgm2ram
                0x9d00ccc8                Base64Decode
                0x9d00d3e0                ultoa
                0x9d00d9ec                strupr
                0x9d00c780                GenerateRandomDWORD
                0x9d00d02c                Base64Encode
 .text          0x9d00db34     0x3d14 ..\Microchip\TCPIP Stack\Objects - TCPIP Demo App-C32\HTTP2.o
                0x9d00db34                HTTPPrint
                0x9d010cbc                HTTPReadPostName
                0x9d00e004                HTTPPrint_
                0x9d010d38                HTTPReadPostValue
                0x9d010a1c                HTTPURLDecode
                0x9d00e15c                HTTPServer
                0x9d011648                HTTPIncFile
                0x9d00e054                HTTPInit
                0x9d010bf0                HTTPGetArg
 .text          0x9d011848      0x5ec ..\Microchip\TCPIP Stack\Objects - TCPIP Demo App-C32\ICMP.o
                0x9d011a30                ICMPSendPing
                0x9d011a8c                ICMPSendPingToHost
                0x9d011dac                ICMPBeginUsage
                0x9d011848                ICMPProcess
                0x9d011e04                ICMPEndUsage
                0x9d011af8                ICMPGetReply
 .text          0x9d011e34      0x31c ..\Microchip\TCPIP Stack\Objects - TCPIP Demo App-C32\IP.o
                0x9d011e34                IPGetHeader
                0x9d011f70                IPPutHeader
                0x9d01207c                IPSetRxBuffer
 .text          0x9d012150      0x48c ..\Microchip\TCPIP Stack\Objects - TCPIP Demo App-C32\LCDBlocking.o
                0x9d01222c                LCDInit
                0x9d012580                LCDErase
                0x9d0123ac                LCDUpdate
 .text          0x9d0125dc     0x1ba4 ..\Microchip\TCPIP Stack\Objects - TCPIP Demo App-C32\MPFS2.o
                0x9d0125dc                MPFSInit
                0x9d0129ac                MPFSOpenID
                0x9d013cac                MPFSGetBytesRem
                0x9d013b14                MPFSGetFlags
                0x9d013164                MPFSSeek
                0x9d013864                MPFSPutEnd
                0x9d013f0c                MPFSGetFilename
                0x9d012e60                MPFSGetArray
                0x9d012bac                MPFSGet
                0x9d01401c                MPFSGetPosition
                0x9d013be0                MPFSGetSize
                0x9d012674                MPFSOpen
                0x9d0136a8                MPFSPutArray
                0x9d01397c                MPFSGetTimestamp
                0x9d0135b0                MPFSFormat
                0x9d014090                MPFSGetID
                0x9d013d58                MPFSGetStartAddr
                0x9d012b40                MPFSClose
                0x9d013a48                MPFSGetMicrotime
                0x9d013e28                MPFSGetEndAddr
                0x9d013110                MPFSGetLong
 .text          0x9d014180      0x6fc ..\Microchip\TCPIP Stack\Objects - TCPIP Demo App-C32\NBNS.o
                0x9d014180                NBNSTask
 .text          0x9d01487c      0x178 ..\Microchip\TCPIP Stack\Objects - TCPIP Demo App-C32\Reboot.o
                0x9d01487c                RebootTask
 .text          0x9d0149f4     0x25c8 ..\Microchip\TCPIP Stack\Objects - TCPIP Demo App-C32\SMTP.o
                0x9d016888                SMTPSendMail
                0x9d016b7c                SMTPPutString
                0x9d0168dc                SMTPIsPutReady
                0x9d014b5c                SMTPTask
                0x9d014a90                SMTPEndUsage
                0x9d0149f4                SMTPBeginUsage
                0x9d016adc                SMTPPutArray
                0x9d016c08                SMTPFlush
                0x9d016938                SMTPPut
                0x9d016c40                SMTPPutDone
                0x9d0168b4                SMTPIsBusy
 .text          0x9d016fbc     0x48b4 ..\Microchip\TCPIP Stack\Objects - TCPIP Demo App-C32\SNMP.o
                0x9d016fbc                SNMPInit
                0x9d017300                SNMPNotify
                0x9d017254                SNMPIsNotifyReady
                0x9d017000                SNMPTask
                0x9d0171a4                SNMPNotifyPrepare
 .text          0x9d01b870      0x4c0 ..\Microchip\TCPIP Stack\Objects - TCPIP Demo App-C32\SNTP.o
                0x9d01bc98                SNTPGetUTCSeconds
                0x9d01b870                SNTPClient
 .text          0x9d01bd30      0x958 ..\Microchip\TCPIP Stack\Objects - TCPIP Demo App-C32\SPIEEPROM.o
                0x9d01c118                XEEWrite
                0x9d01bdfc                XEERead
                0x9d01c530                XEEIsBusy
                0x9d01c234                XEEEndWrite
                0x9d01bd30                XEEInit
                0x9d01bea8                XEEReadArray
                0x9d01c1b4                XEEWriteArray
                0x9d01bdc8                XEEBeginRead
                0x9d01c0e4                XEEBeginWrite
                0x9d01be84                XEEEndRead
 .text          0x9d01c688      0x408 ..\Microchip\TCPIP Stack\Objects - TCPIP Demo App-C32\StackTsk.o
                0x9d01c744                StackTask
                0x9d01c688                StackInit
                0x9d01ca08                StackApplications
 .text          0x9d01ca90     0x8134 ..\Microchip\TCPIP Stack\Objects - TCPIP Demo App-C32\TCP.o
                0x9d01e130                TCPGetTxFIFOFull
                0x9d01cec4                TCPOpen
                0x9d01e28c                TCPIsGetReady
                0x9d01d700                TCPIsPutReady
                0x9d01d5fc                TCPGetRemoteInfo
                0x9d01d3d4                TCPIsConnected
                0x9d01f15c                TCPFindEx
                0x9d01d678                TCPFlush
                0x9d01e428                TCPGet
                0x9d0201f0                TCPProcess
                0x9d01d430                TCPDisconnect
                0x9d01ea90                TCPGetRxFIFOFree
                0x9d01d8f4                TCPPut
                0x9d01dc48                TCPPutArray
                0x9d01e6b0                TCPGetArray
                0x9d01e0cc                TCPPutString
                0x9d01f1d0                TCPTick
                0x9d02426c                TCPAdjustFIFOSize
                0x9d01eb40                TCPFindArrayEx
                0x9d01d328                TCPWasReset
                0x9d01e1e4                TCPDiscard
                0x9d01cbc4                TCPInit
 .text          0x9d024bc4      0x5b0 ..\Microchip\TCPIP Stack\Objects - TCPIP Demo App-C32\TCPPerformanceTest.o
                0x9d024f40                TCPRXPerformanceTask
                0x9d024bfc                TCPTXPerformanceTask
                0x9d024bc4                TCPPerformanceTask
 .text          0x9d025174      0xc14 ..\Microchip\TCPIP Stack\Objects - TCPIP Demo App-C32\Telnet.o
                0x9d025174                TelnetTask
 .text          0x9d025d88      0x304 ..\Microchip\TCPIP Stack\Objects - TCPIP Demo App-C32\Tick.o
                0x9d025d88                TickInit
                0x9d025f08                TickGetDiv256
                0x9d025f5c                TickGetDiv64K
                0x9d025fb0                TickConvertToMilliseconds
                0x9d025ed4                TickGet
                0x9d026008                _T1Interrupt
 .text          0x9d02608c      0x734 ..\Microchip\TCPIP Stack\Objects - TCPIP Demo App-C32\UART2TCPBridge.o
                0x9d026504                _U2RXInterrupt
                0x9d026108                UART2TCPBridgeTask
                0x9d026670                U2Interrupt
                0x9d02608c                UART2TCPBridgeInit
                0x9d0265c8                _U2TXInterrupt
 .text          0x9d0267c0       0xcc ..\Microchip\TCPIP Stack\Objects - TCPIP Demo App-C32\UART.o
                0x9d0267c0                ReadStringUART
 .text          0x9d02688c      0xc90 ..\Microchip\TCPIP Stack\Objects - TCPIP Demo App-C32\UDP.o
                0x9d027004                UDPGet
                0x9d0268f8                UDPTask
                0x9d026d68                UDPPutString
                0x9d027094                UDPGetArray
                0x9d02688c                UDPInit
                0x9d026b00                UDPSetTxBuffer
                0x9d026f68                UDPIsGetReady
                0x9d027160                UDPDiscard
                0x9d026b50                UDPSetRxBuffer
                0x9d026920                UDPOpen
                0x9d026ba0                UDPIsPutReady
                0x9d026dbc                UDPFlush
                0x9d026c34                UDPPut
                0x9d026cc4                UDPPutArray
                0x9d026a74                UDPClose
                0x9d0271bc                UDPProcess
 .text          0x9d02751c     0x15e0 Objects - TCPIP Demo App-C32\CustomSNMPApp.o
                0x9d0276f0                SNMPTrapDemo
                0x9d027db0                SNMPIsValidSetLen
                0x9d027e58                SNMPSetVar
                0x9d028348                SNMPGetVar
                0x9d027c0c                SNMPValidateCommunity
                0x9d028270                SNMPGetNextIndex
                0x9d027954                SNMPSendTrap
 .text          0x9d028afc      0x4d8 Objects - TCPIP Demo App-C32\UARTConfig.o
                0x9d028afc                DoUARTConfig
 .text          0x9d028fd4      0x320 Objects - TCPIP Demo App-C32\GenericTCPClient.o
                0x9d028fd4                GenericTCPClient
 .text          0x9d0292f4      0x210 Objects - TCPIP Demo App-C32\GenericTCPServer.o
                0x9d0292f4                GenericTCPServer
 .text          0x9d029504      0x1e8 Objects - TCPIP Demo App-C32\PingDemo.o
                0x9d029504                PingDemo
 .text          0x9d0296ec      0x2dc Objects - TCPIP Demo App-C32\SMTPDemo.o
                0x9d0296ec                SMTPDemo
 .text          0x9d0299c8     0x176c ..\Microchip\TCPIP Stack\Objects - TCPIP Demo App-C32\BerkeleyAPI.o
                0x9d02aa8c                recv
                0x9d02a1dc                connect
                0x9d02ad5c                recvfrom
                0x9d029a70                socket
                0x9d02a4c4                send
                0x9d029f6c                accept
                0x9d029bb4                bind
                0x9d02a7c8                sendto
                0x9d029cd4                listen
                0x9d02af28                gethostname
                0x9d02b02c                closesocket
                0x9d0299c8                BerkeleySocketInit
 .text          0x9d02b134      0x454 Objects - TCPIP Demo App-C32\BerkeleyUDPClientDemo.o
                0x9d02b4f0                BerkeleySNTPGetUTCSeconds
                0x9d02b134                BerkeleyUDPClientDemo
 .text          0x9d02b588      0x298 Objects - TCPIP Demo App-C32\BerkeleyTCPClientDemo.o
                0x9d02b588                BerkeleyTCPClientDemo
 .text          0x9d02b820      0x31c Objects - TCPIP Demo App-C32\BerkeleyTCPServerDemo.o
                0x9d02b820                BerkeleyTCPServerDemo
 .text          0x9d02bb3c      0x44c C:/Program Files/Microchip/MPLAB C32 Suite/bin/../lib/gcc/pic32mx/3.4.4/size\libgcc.a(_udivdi3.o)
                0x9d02bb3c                __udivdi3
 .text          0x9d02bf88       0x98 C:/Program Files/Microchip/MPLAB C32 Suite/bin/../lib/gcc/pic32mx/3.4.4/../../../../pic32mx/lib/size\libc.a(memcmp.o)
                0x9d02bf88                memcmp
 .text          0x9d02c020      0x168 C:/Program Files/Microchip/MPLAB C32 Suite/bin/../lib/gcc/pic32mx/3.4.4/../../../../pic32mx/lib/size\libc.a(memcpy.o)
                0x9d02c020                memcpy
 .text          0x9d02c188       0xa8 C:/Program Files/Microchip/MPLAB C32 Suite/bin/../lib/gcc/pic32mx/3.4.4/../../../../pic32mx/lib/size\libc.a(memset.o)
                0x9d02c188                memset
 .text          0x9d02c230      0x120 C:/Program Files/Microchip/MPLAB C32 Suite/bin/../lib/gcc/pic32mx/3.4.4/../../../../pic32mx/lib/size\libc.a(strcmp.o)
                0x9d02c230                strcmp
 .text          0x9d02c350      0x1a0 C:/Program Files/Microchip/MPLAB C32 Suite/bin/../lib/gcc/pic32mx/3.4.4/../../../../pic32mx/lib/size\libc.a(strcpy.o)
                0x9d02c350                strcpy
 .text          0x9d02c4f0      0x168 C:/Program Files/Microchip/MPLAB C32 Suite/bin/../lib/gcc/pic32mx/3.4.4/../../../../pic32mx/lib/size\libc.a(strlen.o)
                0x9d02c4f0                strlen
 .text.general_exception
                0x9d02c658       0xd0 C:/Program Files/Microchip/MPLAB C32 Suite/bin/../lib/gcc/pic32mx/3.4.4/../../../../pic32mx/lib/size\libc.a(general-exception.o)
                0x9d02c658                _general_exception_context
 .text.strcat   0x9d02c728       0x9c C:/Program Files/Microchip/MPLAB C32 Suite/bin/../lib/gcc/pic32mx/3.4.4/../../../../pic32mx/lib/size\libc.a(strcat.o)
                0x9d02c728                strcat
 .text.strncmp  0x9d02c7c4       0xd8 C:/Program Files/Microchip/MPLAB C32 Suite/bin/../lib/gcc/pic32mx/3.4.4/../../../../pic32mx/lib/size\libc.a(strncmp.o)
                0x9d02c7c4                strncmp
 .text.strchr   0x9d02c89c       0x90 C:/Program Files/Microchip/MPLAB C32 Suite/bin/../lib/gcc/pic32mx/3.4.4/../../../../pic32mx/lib/size\libc.a(strchr.o)
                0x9d02c89c                strchr
 .text.strstr   0x9d02c92c       0x50 C:/Program Files/Microchip/MPLAB C32 Suite/bin/../lib/gcc/pic32mx/3.4.4/../../../../pic32mx/lib/size\libc.a(strstr.o)
                0x9d02c92c                strstr
 .text.exit     0x9d02c97c       0x9c C:/Program Files/Microchip/MPLAB C32 Suite/bin/../lib/gcc/pic32mx/3.4.4/../../../../pic32mx/lib/size\libc.a(exit.o)
                0x9d02c97c                exit
 .text.rand_r   0x9d02ca18       0x28 C:/Program Files/Microchip/MPLAB C32 Suite/bin/../lib/gcc/pic32mx/3.4.4/../../../../pic32mx/lib/size\libc.a(rand.o)
                0x9d02ca18                rand_r
 .text.rand     0x9d02ca40       0x4c C:/Program Files/Microchip/MPLAB C32 Suite/bin/../lib/gcc/pic32mx/3.4.4/../../../../pic32mx/lib/size\libc.a(rand.o)
                0x9d02ca40                rand
 .text.srand    0x9d02ca8c       0x44 C:/Program Files/Microchip/MPLAB C32 Suite/bin/../lib/gcc/pic32mx/3.4.4/../../../../pic32mx/lib/size\libc.a(rand.o)
                0x9d02ca8c                srand
 .text.atol     0x9d02cad0       0x20 C:/Program Files/Microchip/MPLAB C32 Suite/bin/../lib/gcc/pic32mx/3.4.4/../../../../pic32mx/lib/size\libc.a(atol.o)
                0x9d02cad0                atol
 .text.atoi     0x9d02caf0       0x20 C:/Program Files/Microchip/MPLAB C32 Suite/bin/../lib/gcc/pic32mx/3.4.4/../../../../pic32mx/lib/size\libc.a(atoi.o)
                0x9d02caf0                atoi
 .text.strtol   0x9d02cb10      0x1ec C:/Program Files/Microchip/MPLAB C32 Suite/bin/../lib/gcc/pic32mx/3.4.4/../../../../pic32mx/lib/size\libc.a(strtol.o)
                0x9d02cb10                strtol
 .text._filbuf_simple
                0x9d02ccfc       0x48 C:/Program Files/Microchip/MPLAB C32 Suite/bin/../lib/gcc/pic32mx/3.4.4/../../../../pic32mx/lib/size\libc.a(_iobfuncs.o)
                0x9d02ccfc                _filbuf_simple
 .text._fflush_simple
                0x9d02cd44       0x6c C:/Program Files/Microchip/MPLAB C32 Suite/bin/../lib/gcc/pic32mx/3.4.4/../../../../pic32mx/lib/size\libc.a(_iobfuncs.o)
                0x9d02cd44                _fflush_simple
 .text._flsbuf_simple
                0x9d02cdb0       0xdc C:/Program Files/Microchip/MPLAB C32 Suite/bin/../lib/gcc/pic32mx/3.4.4/../../../../pic32mx/lib/size\libc.a(_iobfuncs.o)
                0x9d02cdb0                _flsbuf_simple
 .text._fwrite_simple
                0x9d02ce8c       0x84 C:/Program Files/Microchip/MPLAB C32 Suite/bin/../lib/gcc/pic32mx/3.4.4/../../../../pic32mx/lib/size\libc.a(_iobfuncs.o)
                0x9d02ce8c                _fwrite_simple
 .text._fsync_simple
                0x9d02cf10       0x34 C:/Program Files/Microchip/MPLAB C32 Suite/bin/../lib/gcc/pic32mx/3.4.4/../../../../pic32mx/lib/size\libc.a(_iobfuncs.o)
                0x9d02cf10                _fsync_simple
 .text._weak_pthread_mutex_init
                0x9d02cf44        0x8 C:/Program Files/Microchip/MPLAB C32 Suite/bin/../lib/gcc/pic32mx/3.4.4/../../../../pic32mx/lib/size\libc.a(stubs.o)
                0x9d02cf44                _weak_pthread_mutex_init
                0x9d02cf44                pthread_mutex_init
 .text._weak_pthread_mutex_destroy
                0x9d02cf4c        0x8 C:/Program Files/Microchip/MPLAB C32 Suite/bin/../lib/gcc/pic32mx/3.4.4/../../../../pic32mx/lib/size\libc.a(stubs.o)
                0x9d02cf4c                _weak_pthread_mutex_destroy
                0x9d02cf4c                pthread_mutex_destroy
 .text._weak_pthread_mutex_lock
                0x9d02cf54        0x8 C:/Program Files/Microchip/MPLAB C32 Suite/bin/../lib/gcc/pic32mx/3.4.4/../../../../pic32mx/lib/size\libc.a(stubs.o)
                0x9d02cf54                _weak_pthread_mutex_lock
                0x9d02cf54                pthread_mutex_lock
 .text._weak_pthread_mutex_trylock
                0x9d02cf5c        0x8 C:/Program Files/Microchip/MPLAB C32 Suite/bin/../lib/gcc/pic32mx/3.4.4/../../../../pic32mx/lib/size\libc.a(stubs.o)
                0x9d02cf5c                _weak_pthread_mutex_trylock
                0x9d02cf5c                pthread_mutex_trylock
 .text._weak_pthread_mutex_unlock
                0x9d02cf64        0x8 C:/Program Files/Microchip/MPLAB C32 Suite/bin/../lib/gcc/pic32mx/3.4.4/../../../../pic32mx/lib/size\libc.a(stubs.o)
                0x9d02cf64                _weak_pthread_mutex_unlock
                0x9d02cf64                pthread_mutex_unlock
 .text._weak_pthread_mutex_setname_np
                0x9d02cf6c        0x8 C:/Program Files/Microchip/MPLAB C32 Suite/bin/../lib/gcc/pic32mx/3.4.4/../../../../pic32mx/lib/size\libc.a(stubs.o)
                0x9d02cf6c                pthread_mutex_setname_np
                0x9d02cf6c                _weak_pthread_mutex_setname_np
 .text._weak_pthread_mutexattr_init
                0x9d02cf74        0x8 C:/Program Files/Microchip/MPLAB C32 Suite/bin/../lib/gcc/pic32mx/3.4.4/../../../../pic32mx/lib/size\libc.a(stubs.o)
                0x9d02cf74                _weak_pthread_mutexattr_init
                0x9d02cf74                pthread_mutexattr_init
 .text._weak_pthread_mutexattr_destroy
                0x9d02cf7c        0x8 C:/Program Files/Microchip/MPLAB C32 Suite/bin/../lib/gcc/pic32mx/3.4.4/../../../../pic32mx/lib/size\libc.a(stubs.o)
                0x9d02cf7c                pthread_mutexattr_destroy
                0x9d02cf7c                _weak_pthread_mutexattr_destroy
 .text._weak_pthread_mutexattr_setname_np
                0x9d02cf84        0x8 C:/Program Files/Microchip/MPLAB C32 Suite/bin/../lib/gcc/pic32mx/3.4.4/../../../../pic32mx/lib/size\libc.a(stubs.o)
                0x9d02cf84                _weak_pthread_mutexattr_setname_np
                0x9d02cf84                pthread_mutexattr_setname_np
 .text._weak_pthread_mutexattr_settype_np
                0x9d02cf8c        0x8 C:/Program Files/Microchip/MPLAB C32 Suite/bin/../lib/gcc/pic32mx/3.4.4/../../../../pic32mx/lib/size\libc.a(stubs.o)
                0x9d02cf8c                _weak_pthread_mutexattr_settype_np
                0x9d02cf8c                pthread_mutexattr_settype_np
 .text._weak_pthread_sysconf_np
                0x9d02cf94        0x8 C:/Program Files/Microchip/MPLAB C32 Suite/bin/../lib/gcc/pic32mx/3.4.4/../../../../pic32mx/lib/size\libc.a(stubs.o)
                0x9d02cf94                _weak_pthread_sysconf_np
                0x9d02cf94                pthread_sysconf_np
 .text._weak_pthread_sigdisable_np
                0x9d02cf9c        0x8 C:/Program Files/Microchip/MPLAB C32 Suite/bin/../lib/gcc/pic32mx/3.4.4/../../../../pic32mx/lib/size\libc.a(stubs.o)
                0x9d02cf9c                _weak_pthread_sigdisable_np
                0x9d02cf9c                pthread_sigdisable_np
 .text._weak_pthread_sigrestore_np
                0x9d02cfa4        0x8 C:/Program Files/Microchip/MPLAB C32 Suite/bin/../lib/gcc/pic32mx/3.4.4/../../../../pic32mx/lib/size\libc.a(stubs.o)
                0x9d02cfa4                pthread_sigrestore_np
                0x9d02cfa4                _weak_pthread_sigrestore_np
 .text._weak__pthread_cleanup_push
                0x9d02cfac        0x8 C:/Program Files/Microchip/MPLAB C32 Suite/bin/../lib/gcc/pic32mx/3.4.4/../../../../pic32mx/lib/size\libc.a(stubs.o)
                0x9d02cfac                _weak__pthread_cleanup_push
                0x9d02cfac                _pthread_cleanup_push
 .text._weak__pthread_cleanup_pop
                0x9d02cfb4        0x8 C:/Program Files/Microchip/MPLAB C32 Suite/bin/../lib/gcc/pic32mx/3.4.4/../../../../pic32mx/lib/size\libc.a(stubs.o)
                0x9d02cfb4                _pthread_cleanup_pop
                0x9d02cfb4                _weak__pthread_cleanup_pop
 .text._weak__pthread_cleanup_push_defer
                0x9d02cfbc        0x8 C:/Program Files/Microchip/MPLAB C32 Suite/bin/../lib/gcc/pic32mx/3.4.4/../../../../pic32mx/lib/size\libc.a(stubs.o)
                0x9d02cfbc                _weak__pthread_cleanup_push_defer
                0x9d02cfbc                _pthread_cleanup_push_defer
 .text._weak__pthread_cleanup_pop_restore
                0x9d02cfc4        0x8 C:/Program Files/Microchip/MPLAB C32 Suite/bin/../lib/gcc/pic32mx/3.4.4/../../../../pic32mx/lib/size\libc.a(stubs.o)
                0x9d02cfc4                _pthread_cleanup_pop_restore
                0x9d02cfc4                _weak__pthread_cleanup_pop_restore
 .text._weak_pthread_once
                0x9d02cfcc       0x2c C:/Program Files/Microchip/MPLAB C32 Suite/bin/../lib/gcc/pic32mx/3.4.4/../../../../pic32mx/lib/size\libc.a(stubs.o)
                0x9d02cfcc                _weak_pthread_once
                0x9d02cfcc                pthread_once
                0x9d02cfcc                _pthread_once
 .text._weak_pthread_key_create
                0x9d02cff8        0x8 C:/Program Files/Microchip/MPLAB C32 Suite/bin/../lib/gcc/pic32mx/3.4.4/../../../../pic32mx/lib/size\libc.a(stubs.o)
                0x9d02cff8                pthread_key_create
                0x9d02cff8                _weak_pthread_key_create
 .text._weak_pthread_setspecific
                0x9d02d000        0x8 C:/Program Files/Microchip/MPLAB C32 Suite/bin/../lib/gcc/pic32mx/3.4.4/../../../../pic32mx/lib/size\libc.a(stubs.o)
                0x9d02d000                _weak_pthread_setspecific
                0x9d02d000                pthread_setspecific
 .text._weak_pthread_getspecific
                0x9d02d008        0x8 C:/Program Files/Microchip/MPLAB C32 Suite/bin/../lib/gcc/pic32mx/3.4.4/../../../../pic32mx/lib/size\libc.a(stubs.o)
                0x9d02d008                pthread_getspecific
                0x9d02d008                _weak_pthread_getspecific
 .text._weak__libc_private_storage
                0x9d02d010        0x8 C:/Program Files/Microchip/MPLAB C32 Suite/bin/../lib/gcc/pic32mx/3.4.4/../../../../pic32mx/lib/size\libc.a(stubs.o)
                0x9d02d010                _libc_private_storage
                0x9d02d010                _weak__libc_private_storage
 .text._bootstrap_exception_handler
                0x9d02d018        0x8 C:/Program Files/Microchip/MPLAB C32 Suite/bin/../lib/gcc/pic32mx/3.4.4/../../../../pic32mx/lib/size\libc.a(default-bootstrap-exception-handler.o)
                0x9d02d018                _bootstrap_exception_handler
 .text._on_reset
                0x9d02d020        0x8 C:/Program Files/Microchip/MPLAB C32 Suite/bin/../lib/gcc/pic32mx/3.4.4/../../../../pic32mx/lib/size\libc.a(default-on-reset.o)
                0x9d02d020                _on_reset
 .text._on_bootstrap
                0x9d02d028        0x8 C:/Program Files/Microchip/MPLAB C32 Suite/bin/../lib/gcc/pic32mx/3.4.4/../../../../pic32mx/lib/size\libc.a(default-on-bootstrap.o)
                0x9d02d028                _on_bootstrap
 .text          0x9d02d030       0x18 C:/Program Files/Microchip/MPLAB C32 Suite/bin/../lib/gcc/pic32mx/3.4.4/../../../../pic32mx/lib/size\libc.a(default-nmi-handler.o)
                0x9d02d030                _nmi_handler
 .text._mon_getc
                0x9d02d048        0x8 C:/Program Files/Microchip/MPLAB C32 Suite/bin/../lib/gcc/pic32mx/3.4.4/../../../../pic32mx/lib/size\libc.a(_mon_getc.o)
                0x9d02d048                _mon_getc
 .text._mon_write
                0x9d02d050       0x4c C:/Program Files/Microchip/MPLAB C32 Suite/bin/../lib/gcc/pic32mx/3.4.4/../../../../pic32mx/lib/size\libc.a(_mon_write.o)
                0x9d02d050                _mon_write
 .text._exit    0x9d02d09c        0x8 C:/Program Files/Microchip/MPLAB C32 Suite/bin/../lib/gcc/pic32mx/3.4.4/../../../../pic32mx/lib/size\libc.a(_exit.o)
                0x9d02d09c                _exit
 .text._mon_putc
                0x9d02d0a4       0x28 C:/Program Files/Microchip/MPLAB C32 Suite/bin/../lib/gcc/pic32mx/3.4.4/../../../../pic32mx/lib/size\libc.a(_mon_putc.o)
                0x9d02d0a4                _mon_putc
 .text.INTDisableInterrupts
                0x9d02d0cc        0x8 C:/Program Files/Microchip/MPLAB C32 Suite/bin/../lib/gcc/pic32mx/3.4.4/../../../../pic32mx/lib/size\libmchp_peripheral.a(int_disable_interrupts_lib.o)
                0x9d02d0cc                INTDisableInterrupts
 .text.INTEnableSystemMultiVectoredInt
                0x9d02d0d4       0x34 C:/Program Files/Microchip/MPLAB C32 Suite/bin/../lib/gcc/pic32mx/3.4.4/../../../../pic32mx/lib/size\libmchp_peripheral.a(int_enable_mv_int_lib.o)
                0x9d02d0d4                INTEnableSystemMultiVectoredInt
 .text.INTRestoreInterrupts
                0x9d02d108       0x1c C:/Program Files/Microchip/MPLAB C32 Suite/bin/../lib/gcc/pic32mx/3.4.4/../../../../pic32mx/lib/size\libmchp_peripheral.a(int_restore_interrupts_lib.o)
                0x9d02d108                INTRestoreInterrupts
 .text.putsUART1
                0x9d02d124       0x50 C:/Program Files/Microchip/MPLAB C32 Suite/bin/../lib/gcc/pic32mx/3.4.4/../../../../pic32mx/lib/size\libmchp_peripheral.a(puts_uartx_lib.o)
                0x9d02d124                putsUART1
 .text.putsUART2
                0x9d02d174       0x50 C:/Program Files/Microchip/MPLAB C32 Suite/bin/../lib/gcc/pic32mx/3.4.4/../../../../pic32mx/lib/size\libmchp_peripheral.a(puts_uartx_lib.o)
                0x9d02d174                putsUART2
 .text.SoftReset
                0x9d02d1c4       0x78 C:/Program Files/Microchip/MPLAB C32 Suite/bin/../lib/gcc/pic32mx/3.4.4/../../../../pic32mx/lib/size\libmchp_peripheral.a(soft_reset_lib.o)
                0x9d02d1c4                SoftReset
 .text.CheKseg0CacheOff
                0x9d02d23c       0x18 C:/Program Files/Microchip/MPLAB C32 Suite/bin/../lib/gcc/pic32mx/3.4.4/../../../../pic32mx/lib/size\libmchp_peripheral.a(pcache.o)
                0x9d02d23c                CheKseg0CacheOff
 .text.CheKseg0CacheOn
                0x9d02d254       0x18 C:/Program Files/Microchip/MPLAB C32 Suite/bin/../lib/gcc/pic32mx/3.4.4/../../../../pic32mx/lib/size\libmchp_peripheral.a(pcache.o)
                0x9d02d254                CheKseg0CacheOn
 .text.INTEnableInterrupts
                0x9d02d26c        0x8 C:/Program Files/Microchip/MPLAB C32 Suite/bin/../lib/gcc/pic32mx/3.4.4/../../../../pic32mx/lib/size\libmchp_peripheral.a(int_enable_interrupts_lib.o)
                0x9d02d26c                INTEnableInterrupts
 *(.text.*personality*)
 *(.gnu.warning)
 *(.mips16.fn.*)
 *(.mips16.call.*)
                0x9d02d274                _text_end = .

.rodata         0x9d02d274     0x1f88
 *(.rodata .rodata.* .gnu.linkonce.r.*)
 .rodata        0x9d02d274       0xd8 Objects - TCPIP Demo App-C32\MainDemo.o
 .rodata        0x9d02d34c      0x618 Objects - TCPIP Demo App-C32\CustomHTTPApp.o
                0x9d02d714                HTML_UP_ARROW
                0x9d02d718                HTML_DOWN_ARROW
 .rodata        0x9d02d964       0x1c ..\Microchip\TCPIP Stack\Objects - TCPIP Demo App-C32\Announce.o
 .rodata        0x9d02d980       0x34 ..\Microchip\TCPIP Stack\Objects - TCPIP Demo App-C32\DHCP.o
 .rodata        0x9d02d9b4       0x20 ..\Microchip\TCPIP Stack\Objects - TCPIP Demo App-C32\DNS.o
 .rodata        0x9d02d9d4      0x21c ..\Microchip\TCPIP Stack\Objects - TCPIP Demo App-C32\DynDNS.o
 .rodata        0x9d02dbf0      0x140 ..\Microchip\TCPIP Stack\Objects - TCPIP Demo App-C32\Hashes.o
 .rodata        0x9d02dd30      0x8cc ..\Microchip\TCPIP Stack\Objects - TCPIP Demo App-C32\HTTP2.o
 .rodata        0x9d02e5fc       0x1c ..\Microchip\TCPIP Stack\Objects - TCPIP Demo App-C32\ICMP.o
 .rodata        0x9d02e618        0x8 ..\Microchip\TCPIP Stack\Objects - TCPIP Demo App-C32\MPFS2.o
 .rodata        0x9d02e620       0x14 ..\Microchip\TCPIP Stack\Objects - TCPIP Demo App-C32\Reboot.o
 .rodata        0x9d02e634      0x1e0 ..\Microchip\TCPIP Stack\Objects - TCPIP Demo App-C32\SMTP.o
 .rodata        0x9d02e814       0x54 ..\Microchip\TCPIP Stack\Objects - TCPIP Demo App-C32\SNMP.o
 .rodata        0x9d02e868       0x44 ..\Microchip\TCPIP Stack\Objects - TCPIP Demo App-C32\SNTP.o
 .rodata        0x9d02e8ac       0xa8 ..\Microchip\TCPIP Stack\Objects - TCPIP Demo App-C32\TCP.o
                0x9d02e8ac                TCPSocketInitializer
 .rodata        0x9d02e954       0x5c ..\Microchip\TCPIP Stack\Objects - TCPIP Demo App-C32\TCPPerformanceTest.o
 .rodata        0x9d02e9b0      0x200 ..\Microchip\TCPIP Stack\Objects - TCPIP Demo App-C32\Telnet.o
 .rodata        0x9d02ebb0       0x2c Objects - TCPIP Demo App-C32\CustomSNMPApp.o
 .rodata        0x9d02ebdc      0x240 Objects - TCPIP Demo App-C32\UARTConfig.o
 .rodata        0x9d02ee1c       0xa8 Objects - TCPIP Demo App-C32\GenericTCPClient.o
 .rodata        0x9d02eec4       0x44 Objects - TCPIP Demo App-C32\PingDemo.o
 .rodata        0x9d02ef08       0x50 Objects - TCPIP Demo App-C32\SMTPDemo.o
 .rodata        0x9d02ef58       0x28 Objects - TCPIP Demo App-C32\BerkeleyUDPClientDemo.o
 .rodata        0x9d02ef80      0x150 Objects - TCPIP Demo App-C32\BerkeleyTCPClientDemo.o
 .rodata        0x9d02f0d0       0x14 Objects - TCPIP Demo App-C32\BerkeleyTCPServerDemo.o
 .rodata        0x9d02f0e4       0x14 C:/Program Files/Microchip/MPLAB C32 Suite/bin/../lib/gcc/pic32mx/3.4.4/../../../../pic32mx/lib/size\libc.a(_iobdata.o)
                0x9d02f0e4                _io_funcs
 .rodata        0x9d02f0f8      0x104 C:/Program Files/Microchip/MPLAB C32 Suite/bin/../lib/gcc/pic32mx/3.4.4/../../../../pic32mx/lib/size\libc.a(ctype.o)
                0x9d02f0f8                _ctype
 *(.rodata1)
                0x9d02f1fc                . = ALIGN (0x4)

.sdata2         0x9d02f1fc        0x0
 *(.sdata2 .sdata2.* .gnu.linkonce.s2.*)
                0x9d02f1fc                . = ALIGN (0x4)

.sbss2          0x9d02f1fc        0x0
 *(.sbss2 .sbss2.* .gnu.linkonce.sb2.*)
                0x9d02f1fc                . = ALIGN (0x4)

.eh_frame_hdr
 *(.eh_frame_hdr)

.eh_frame       0x9d02f1fc       0x20
 *(.eh_frame)
 .eh_frame      0x9d02f1fc       0x20 C:/Program Files/Microchip/MPLAB C32 Suite/bin/../lib/gcc/pic32mx/3.4.4/size\libgcc.a(_udivdi3.o)

.dbg_data       0xa0000000        0x0
                0xa0000000                . = (. + DEFINED (_DEBUGGER)?0x200:0x0)

.data           0xa0000000      0x2f8 load address 0x9d02f21c
                0xa0000000                _data_begin = .
 *(.data .data.* .gnu.linkonce.d.*)
 .data          0xa0000000       0x40 ..\Microchip\TCPIP Stack\Objects - TCPIP Demo App-C32\DynDNS.o
                0xa0000034                ddnsServiceHosts
 .data          0xa0000040       0xa0 ..\Microchip\TCPIP Stack\Objects - TCPIP Demo App-C32\HTTP2.o
 .data          0xa00000e0       0x2c Objects - TCPIP Demo App-C32\CustomSNMPApp.o
                0xa00000e0                trapInfo
 .data          0xa000010c       0x10 Objects - TCPIP Demo App-C32\GenericTCPClient.o
 .data          0xa000011c       0x48 Objects - TCPIP Demo App-C32\SMTPDemo.o
 .data          0xa0000164       0x70 Objects - TCPIP Demo App-C32\BerkeleyTCPClientDemo.o
 .data          0xa00001d4       0x20 C:/Program Files/Microchip/MPLAB C32 Suite/bin/../lib/gcc/pic32mx/3.4.4/../../../../pic32mx/lib/size\libc.a(exit.o)
                0xa00001d4                __exfun_mx
 .data          0xa00001f4       0x30 C:/Program Files/Microchip/MPLAB C32 Suite/bin/../lib/gcc/pic32mx/3.4.4/../../../../pic32mx/lib/size\libc.a(rand.o)
 .data          0xa0000224       0xd4 C:/Program Files/Microchip/MPLAB C32 Suite/bin/../lib/gcc/pic32mx/3.4.4/../../../../pic32mx/lib/size\libc.a(_iobdata.o)
 *(.gnu.linkonce.d.*personality*)
 *(.data1)
                0x9d02f21c                _data_image_begin = LOADADDR (.data)

.eh_frame
 *(.eh_frame)
                0xa00082f0                _gp = (ALIGN (0x10) + 0x7ff0)

.got
 *(.got.plt)
 *(.got)

.sdata          0xa00002f8       0x5c load address 0x9d02f514
                0xa00002f8                _sdata_begin = .
 *(.sdata .sdata.* .gnu.linkonce.s.*)
 .sdata         0xa00002f8        0x8 Objects - TCPIP Demo App-C32\MainDemo.o
                0xa00002f8                myDHCPBindCount
                0xa00002fc                __C30_UART
 .sdata         0xa0000300        0x8 ..\Microchip\TCPIP Stack\Objects - TCPIP Demo App-C32\DHCP.o
                0xa0000300                smDHCPState
 .sdata         0xa0000308        0x4 ..\Microchip\TCPIP Stack\Objects - TCPIP Demo App-C32\DHCPs.o
                0xa0000308                bDHCPServerEnabled
 .sdata         0xa000030c        0x8 ..\Microchip\TCPIP Stack\Objects - TCPIP Demo App-C32\DNS.o
 .sdata         0xa0000314        0x1 ..\Microchip\TCPIP Stack\Objects - TCPIP Demo App-C32\DynDNS.o
 .sdata         0xa0000315        0x1 ..\Microchip\TCPIP Stack\Objects - TCPIP Demo App-C32\Reboot.o
 .sdata         0xa0000316        0x1 ..\Microchip\TCPIP Stack\Objects - TCPIP Demo App-C32\SMTP.o
 .sdata         0xa0000317        0x1 ..\Microchip\TCPIP Stack\Objects - TCPIP Demo App-C32\SNMP.o
 .sdata         0xa0000318        0x2 ..\Microchip\TCPIP Stack\Objects - TCPIP Demo App-C32\TCP.o
 .sdata         0xa000031a        0x2 ..\Microchip\TCPIP Stack\Objects - TCPIP Demo App-C32\TCPPerformanceTest.o
 .sdata         0xa000031c       0x14 ..\Microchip\TCPIP Stack\Objects - TCPIP Demo App-C32\UART2TCPBridge.o
 .sdata         0xa0000330        0x2 ..\Microchip\TCPIP Stack\Objects - TCPIP Demo App-C32\UDP.o
 .sdata         0xa0000332        0x2 Objects - TCPIP Demo App-C32\CustomSNMPApp.o
                0xa0000332                gOIDCorrespondingSnmpMibID
                0xa0000333                gGenericTrapNotification
 .sdata         0xa0000334        0x8 Objects - TCPIP Demo App-C32\GenericTCPClient.o
 .sdata         0xa000033c        0x2 ..\Microchip\TCPIP Stack\Objects - TCPIP Demo App-C32\BerkeleyAPI.o
 .sdata         0xa000033e        0x1 Objects - TCPIP Demo App-C32\BerkeleyUDPClientDemo.o
 *fill*         0xa000033f        0x1 00
 .sdata         0xa0000340        0x8 Objects - TCPIP Demo App-C32\BerkeleyTCPClientDemo.o
 .sdata         0xa0000348        0x8 Objects - TCPIP Demo App-C32\BerkeleyTCPServerDemo.o
 .sdata         0xa0000350        0x4 C:/Program Files/Microchip/MPLAB C32 Suite/bin/../lib/gcc/pic32mx/3.4.4/../../../../pic32mx/lib/size\libc.a(_iobdata.o)
                0xa0000350                _libc_data
                0xa0000354                _sdata_end = .

.lit8
 *(.lit8)

.lit4
 *(.lit4)
                0xa0000354                . = ALIGN (0x4)
                0xa0000354                _data_end = .
                0xa0000354                _bss_begin = .

.sbss           0xa0000354      0x20e
                0xa0000354                _sbss_begin = .
 *(.dynsbss)
 *(.sbss .sbss.* .gnu.linkonce.sb.*)
 .sbss          0xa0000354        0x4 Objects - TCPIP Demo App-C32\MainDemo.o
 .sbss          0xa0000358       0x14 Objects - TCPIP Demo App-C32\CustomHTTPApp.o
 .sbss          0xa000036c        0x8 ..\Microchip\TCPIP Stack\Objects - TCPIP Demo App-C32\Announce.o
 .sbss          0xa0000374        0x4 ..\Microchip\TCPIP Stack\Objects - TCPIP Demo App-C32\ARP.o
 .sbss          0xa0000378       0x28 ..\Microchip\TCPIP Stack\Objects - TCPIP Demo App-C32\DHCP.o
                0xa0000379                DHCPBindCount
                0xa0000378                DHCPFlags
 .sbss          0xa00003a0        0xc ..\Microchip\TCPIP Stack\Objects - TCPIP Demo App-C32\DHCPs.o
 .sbss          0xa00003ac       0x18 ..\Microchip\TCPIP Stack\Objects - TCPIP Demo App-C32\DNS.o
 .sbss          0xa00003c4       0x24 ..\Microchip\TCPIP Stack\Objects - TCPIP Demo App-C32\DynDNS.o
 .sbss          0xa00003e8       0x10 ..\Microchip\TCPIP Stack\Objects - TCPIP Demo App-C32\ENC28J60.o
 .sbss          0xa00003f8        0xc ..\Microchip\TCPIP Stack\Objects - TCPIP Demo App-C32\ICMP.o
 .sbss          0xa0000404        0x4 ..\Microchip\TCPIP Stack\Objects - TCPIP Demo App-C32\IP.o
 .sbss          0xa0000408        0x8 ..\Microchip\TCPIP Stack\Objects - TCPIP Demo App-C32\MPFS2.o
 .sbss          0xa0000410        0x8 ..\Microchip\TCPIP Stack\Objects - TCPIP Demo App-C32\NBNS.o
 .sbss          0xa0000418       0x38 ..\Microchip\TCPIP Stack\Objects - TCPIP Demo App-C32\SMTP.o
 .sbss          0xa0000450       0x1c ..\Microchip\TCPIP Stack\Objects - TCPIP Demo App-C32\SNMP.o
 .sbss          0xa000046c       0x14 ..\Microchip\TCPIP Stack\Objects - TCPIP Demo App-C32\SNTP.o
 .sbss          0xa0000480        0x8 ..\Microchip\TCPIP Stack\Objects - TCPIP Demo App-C32\SPIEEPROM.o
 .sbss          0xa0000488        0x4 ..\Microchip\TCPIP Stack\Objects - TCPIP Demo App-C32\StackTsk.o
 .sbss          0xa000048c        0x2 ..\Microchip\TCPIP Stack\Objects - TCPIP Demo App-C32\TCP.o
 *fill*         0xa000048e        0x2 00
 .sbss          0xa0000490       0x14 ..\Microchip\TCPIP Stack\Objects - TCPIP Demo App-C32\TCPPerformanceTest.o
 .sbss          0xa00004a4       0x10 ..\Microchip\TCPIP Stack\Objects - TCPIP Demo App-C32\Telnet.o
 .sbss          0xa00004b4        0xc ..\Microchip\TCPIP Stack\Objects - TCPIP Demo App-C32\Tick.o
 .sbss          0xa00004c0        0x4 ..\Microchip\TCPIP Stack\Objects - TCPIP Demo App-C32\UART2TCPBridge.o
 .sbss          0xa00004c4        0xc ..\Microchip\TCPIP Stack\Objects - TCPIP Demo App-C32\UDP.o
 .sbss          0xa00004d0       0x30 Objects - TCPIP Demo App-C32\CustomSNMPApp.o
                0xa00004d0                gSendTrapFlag
                0xa00004d1                gSpecificTrapNotification
 .sbss          0xa0000500        0x4 Objects - TCPIP Demo App-C32\GenericTCPClient.o
 .sbss          0xa0000504        0x8 Objects - TCPIP Demo App-C32\GenericTCPServer.o
 .sbss          0xa000050c        0x8 Objects - TCPIP Demo App-C32\PingDemo.o
 .sbss          0xa0000514        0x8 Objects - TCPIP Demo App-C32\SMTPDemo.o
 .sbss          0xa000051c        0xc ..\Microchip\TCPIP Stack\Objects - TCPIP Demo App-C32\BerkeleyAPI.o
 .sbss          0xa0000528       0x10 Objects - TCPIP Demo App-C32\BerkeleyUDPClientDemo.o
 .sbss          0xa0000538        0x8 Objects - TCPIP Demo App-C32\BerkeleyTCPServerDemo.o
 .sbss          0xa0000540        0x4 C:/Program Files/Microchip/MPLAB C32 Suite/bin/../lib/gcc/pic32mx/3.4.4/../../../../pic32mx/lib/size\libc.a(errno.o)
                0xa0000540                errno
 *(.scommon)
 .scommon       0xa0000544        0x8 Objects - TCPIP Demo App-C32\MainDemo.o
                0xa0000544                AN0String
 .scommon       0xa000054c        0x1 ..\Microchip\TCPIP Stack\Objects - TCPIP Demo App-C32\HTTP2.o
                0xa000054c                curHTTPID
 *fill*         0xa000054d        0x3 00
 .scommon       0xa0000550        0x4 ..\Microchip\TCPIP Stack\Objects - TCPIP Demo App-C32\MPFS2.o
                0xa0000550                lastRead
 .scommon       0xa0000554        0x8 ..\Microchip\TCPIP Stack\Objects - TCPIP Demo App-C32\SNMP.o
                0xa0000554                snmpReqVarErrStatus
 .scommon       0xa000055c        0x6 ..\Microchip\TCPIP Stack\Objects - TCPIP Demo App-C32\UDP.o
                0xa000055c                UDPTxCount
                0xa000055e                activeUDPSocket
                0xa0000560                UDPRxCount
                0xa0000562                _sbss_end = .

.bss            0xa0000564      0x860
 *(.dynbss)
 *(.bss .bss.* .gnu.linkonce.b.*)
 .bss           0xa0000564       0xc0 Objects - TCPIP Demo App-C32\CustomHTTPApp.o
 .bss           0xa0000624       0x18 ..\Microchip\TCPIP Stack\Objects - TCPIP Demo App-C32\ARP.o
 .bss           0xa000063c        0xc ..\Microchip\TCPIP Stack\Objects - TCPIP Demo App-C32\DNS.o
 .bss           0xa0000648       0x10 ..\Microchip\TCPIP Stack\Objects - TCPIP Demo App-C32\DynDNS.o
 .bss           0xa0000658        0xc ..\Microchip\TCPIP Stack\Objects - TCPIP Demo App-C32\ICMP.o
 .bss           0xa0000664       0x78 ..\Microchip\TCPIP Stack\Objects - TCPIP Demo App-C32\MPFS2.o
 .bss           0xa00006dc       0x10 ..\Microchip\TCPIP Stack\Objects - TCPIP Demo App-C32\SNMP.o
 .bss           0xa00006ec        0xc ..\Microchip\TCPIP Stack\Objects - TCPIP Demo App-C32\SNTP.o
 .bss           0xa00006f8       0x20 ..\Microchip\TCPIP Stack\Objects - TCPIP Demo App-C32\SPIEEPROM.o
 .bss           0xa0000718      0x224 ..\Microchip\TCPIP Stack\Objects - TCPIP Demo App-C32\TCP.o
 .bss           0xa000093c        0xc ..\Microchip\TCPIP Stack\Objects - TCPIP Demo App-C32\TCPPerformanceTest.o
 .bss           0xa0000948       0x58 ..\Microchip\TCPIP Stack\Objects - TCPIP Demo App-C32\UART2TCPBridge.o
 .bss           0xa00009a0       0x8c ..\Microchip\TCPIP Stack\Objects - TCPIP Demo App-C32\BerkeleyAPI.o
 .bss           0xa0000a2c       0x1c Objects - TCPIP Demo App-C32\BerkeleyUDPClientDemo.o
 .bss           0xa0000a48       0x10 Objects - TCPIP Demo App-C32\BerkeleyTCPClientDemo.o
 .bss           0xa0000a58       0x10 Objects - TCPIP Demo App-C32\BerkeleyTCPServerDemo.o
 .bss           0xa0000a68       0x88 C:/Program Files/Microchip/MPLAB C32 Suite/bin/../lib/gcc/pic32mx/3.4.4/../../../../pic32mx/lib/size\libc.a(_iobdata.o)
 .bss           0xa0000af0       0x80 C:/Program Files/Microchip/MPLAB C32 Suite/bin/../lib/gcc/pic32mx/3.4.4/../../../../pic32mx/lib/size\libc.a(_iobfuncs.o)
 .bss           0xa0000b70        0x4 C:/Program Files/Microchip/MPLAB C32 Suite/bin/../lib/gcc/pic32mx/3.4.4/../../../../pic32mx/lib/size\libc.a(stubs.o)
                0xa0000b70                __isthreaded
 *(COMMON)
 COMMON         0xa0000b74       0x69 Objects - TCPIP Demo App-C32\MainDemo.o
                0xa0000b74                AppConfig
 *fill*         0xa0000bdd        0x3 00
 COMMON         0xa0000be0       0x20 ..\Microchip\TCPIP Stack\Objects - TCPIP Demo App-C32\DynDNS.o
                0xa0000be0                DDNSClient
 COMMON         0xa0000c00       0x40 ..\Microchip\TCPIP Stack\Objects - TCPIP Demo App-C32\Hashes.o
                0xa0000c00                lastBlock
 COMMON         0xa0000c40       0x9c ..\Microchip\TCPIP Stack\Objects - TCPIP Demo App-C32\HTTP2.o
                0xa0000c40                curHTTP
                0xa0000ccc                httpStubs
 COMMON         0xa0000cdc       0x21 ..\Microchip\TCPIP Stack\Objects - TCPIP Demo App-C32\LCDBlocking.o
                0xa0000cdc                LCDText
 *fill*         0xa0000cfd        0x3 00
 COMMON         0xa0000d00       0x2c ..\Microchip\TCPIP Stack\Objects - TCPIP Demo App-C32\SMTP.o
                0xa0000d00                SMTPClient
 COMMON         0xa0000d2c        0xa ..\Microchip\TCPIP Stack\Objects - TCPIP Demo App-C32\StackTsk.o
                0xa0000d2c                remoteNode
 *fill*         0xa0000d36        0x2 00
 COMMON         0xa0000d38       0x8c ..\Microchip\TCPIP Stack\Objects - TCPIP Demo App-C32\UDP.o
                0xa0000d38                UDPSocketInfo
                0xa0000dc4                . = ALIGN (0x4)
                0xa0000dc4                . = ALIGN (0x4)
                0xa0000dc4                _end = .
                0xa0000dc4                _bss_end = .

.heap           0xa0000dc4        0x0
                0xa0000dc4                _heap = .
                0xa0000dc4                . = (. + _min_heap_size)

.stack          0xa0000dc4      0x400
                0xa00011c4                . = (. + _min_stack_size)
 *fill*         0xa0000dc4      0x400 00

.ramfunc        0xa0001800        0x0 load address 0x9d02f570
                0xa0001800                _ramfunc_begin = .
 *(.ramfunc .ramfunc.*)
                0xa0001800                . = ALIGN (0x4)
                0xa0001800                _ramfunc_end = .
                0x9d02f570                _ramfunc_image_begin = LOADADDR (.ramfunc)
                0x00000000                _ramfunc_length = SIZEOF (.ramfunc)
                0x00001800                _bmxdkpba_address = (_ramfunc_begin - 0xa0000000)
                0x00008000                _bmxdudba_address = 0x8000
                0x00008000                _bmxdupba_address = 0x8000
                0xa0008000                _stack = (_ramfunc_length > 0x0)?(_ramfunc_begin - 0x4):0xa0008000
                0x00000001                ASSERT (((_min_stack_size + _min_heap_size) <= (_stack - _heap)), Not enough space to allocate both stack and heap.  Reduce heap and/or stack size.)

.pdr            0x00000000     0x33e0
 *(.pdr)
 .pdr           0x00000000       0xa0 C:/Program Files/Microchip/MPLAB C32 Suite/bin/../lib/gcc/pic32mx/3.4.4/../../../../pic32mx/lib/size/crt0.o
 .pdr           0x000000a0       0xe0 Objects - TCPIP Demo App-C32\MainDemo.o
 .pdr           0x00000180      0x560 Objects - TCPIP Demo App-C32\CustomHTTPApp.o
 .pdr           0x000006e0       0x40 ..\Microchip\TCPIP Stack\Objects - TCPIP Demo App-C32\Announce.o
 .pdr           0x00000720       0xc0 ..\Microchip\TCPIP Stack\Objects - TCPIP Demo App-C32\ARP.o
 .pdr           0x000007e0       0x40 ..\Microchip\TCPIP Stack\Objects - TCPIP Demo App-C32\Delay.o
 .pdr           0x00000820       0xc0 ..\Microchip\TCPIP Stack\Objects - TCPIP Demo App-C32\DHCP.o
 .pdr           0x000008e0       0x60 ..\Microchip\TCPIP Stack\Objects - TCPIP Demo App-C32\DHCPs.o
 .pdr           0x00000940       0xc0 ..\Microchip\TCPIP Stack\Objects - TCPIP Demo App-C32\DNS.o
 .pdr           0x00000a00       0xc0 ..\Microchip\TCPIP Stack\Objects - TCPIP Demo App-C32\DynDNS.o
 .pdr           0x00000ac0      0x400 ..\Microchip\TCPIP Stack\Objects - TCPIP Demo App-C32\ENC28J60.o
 .pdr           0x00000ec0       0xa0 ..\Microchip\TCPIP Stack\Objects - TCPIP Demo App-C32\Hashes.o
 .pdr           0x00000f60      0x1e0 ..\Microchip\TCPIP Stack\Objects - TCPIP Demo App-C32\Helpers.o
 .pdr           0x00001140      0x240 ..\Microchip\TCPIP Stack\Objects - TCPIP Demo App-C32\HTTP2.o
 .pdr           0x00001380       0xc0 ..\Microchip\TCPIP Stack\Objects - TCPIP Demo App-C32\ICMP.o
 .pdr           0x00001440       0x80 ..\Microchip\TCPIP Stack\Objects - TCPIP Demo App-C32\IP.o
 .pdr           0x000014c0       0x80 ..\Microchip\TCPIP Stack\Objects - TCPIP Demo App-C32\LCDBlocking.o
 .pdr           0x00001540      0x2e0 ..\Microchip\TCPIP Stack\Objects - TCPIP Demo App-C32\MPFS2.o
 .pdr           0x00001820       0x60 ..\Microchip\TCPIP Stack\Objects - TCPIP Demo App-C32\NBNS.o
 .pdr           0x00001880       0x20 ..\Microchip\TCPIP Stack\Objects - TCPIP Demo App-C32\Reboot.o
 .pdr           0x000018a0      0x1a0 ..\Microchip\TCPIP Stack\Objects - TCPIP Demo App-C32\SMTP.o
 .pdr           0x00001a40      0x3e0 ..\Microchip\TCPIP Stack\Objects - TCPIP Demo App-C32\SNMP.o
 .pdr           0x00001e20       0x40 ..\Microchip\TCPIP Stack\Objects - TCPIP Demo App-C32\SNTP.o
 .pdr           0x00001e60      0x160 ..\Microchip\TCPIP Stack\Objects - TCPIP Demo App-C32\SPIEEPROM.o
 .pdr           0x00001fc0       0x60 ..\Microchip\TCPIP Stack\Objects - TCPIP Demo App-C32\StackTsk.o
 .pdr           0x00002020      0x3a0 ..\Microchip\TCPIP Stack\Objects - TCPIP Demo App-C32\TCP.o
 .pdr           0x000023c0       0x60 ..\Microchip\TCPIP Stack\Objects - TCPIP Demo App-C32\TCPPerformanceTest.o
 .pdr           0x00002420       0x20 ..\Microchip\TCPIP Stack\Objects - TCPIP Demo App-C32\Telnet.o
 .pdr           0x00002440      0x100 ..\Microchip\TCPIP Stack\Objects - TCPIP Demo App-C32\Tick.o
 .pdr           0x00002540       0xc0 ..\Microchip\TCPIP Stack\Objects - TCPIP Demo App-C32\UART2TCPBridge.o
 .pdr           0x00002600       0x20 ..\Microchip\TCPIP Stack\Objects - TCPIP Demo App-C32\UART.o
 .pdr           0x00002620      0x220 ..\Microchip\TCPIP Stack\Objects - TCPIP Demo App-C32\UDP.o
 .pdr           0x00002840      0x120 Objects - TCPIP Demo App-C32\CustomSNMPApp.o
 .pdr           0x00002960       0x20 Objects - TCPIP Demo App-C32\UARTConfig.o
 .pdr           0x00002980       0x20 Objects - TCPIP Demo App-C32\GenericTCPClient.o
 .pdr           0x000029a0       0x20 Objects - TCPIP Demo App-C32\GenericTCPServer.o
 .pdr           0x000029c0       0x20 Objects - TCPIP Demo App-C32\PingDemo.o
 .pdr           0x000029e0       0x20 Objects - TCPIP Demo App-C32\SMTPDemo.o
 .pdr           0x00002a00      0x180 ..\Microchip\TCPIP Stack\Objects - TCPIP Demo App-C32\BerkeleyAPI.o
 .pdr           0x00002b80       0x40 Objects - TCPIP Demo App-C32\BerkeleyUDPClientDemo.o
 .pdr           0x00002bc0       0x20 Objects - TCPIP Demo App-C32\BerkeleyTCPClientDemo.o
 .pdr           0x00002be0       0x20 Objects - TCPIP Demo App-C32\BerkeleyTCPServerDemo.o
 .pdr           0x00002c00       0x20 C:/Program Files/Microchip/MPLAB C32 Suite/bin/../lib/gcc/pic32mx/3.4.4/size\libgcc.a(_udivdi3.o)
 .pdr           0x00002c20       0x20 C:/Program Files/Microchip/MPLAB C32 Suite/bin/../lib/gcc/pic32mx/3.4.4/../../../../pic32mx/lib/size\libc.a(memcmp.o)
 .pdr           0x00002c40       0x20 C:/Program Files/Microchip/MPLAB C32 Suite/bin/../lib/gcc/pic32mx/3.4.4/../../../../pic32mx/lib/size\libc.a(memcpy.o)
 .pdr           0x00002c60       0x20 C:/Program Files/Microchip/MPLAB C32 Suite/bin/../lib/gcc/pic32mx/3.4.4/../../../../pic32mx/lib/size\libc.a(memset.o)
 .pdr           0x00002c80       0x20 C:/Program Files/Microchip/MPLAB C32 Suite/bin/../lib/gcc/pic32mx/3.4.4/../../../../pic32mx/lib/size\libc.a(strcmp.o)
 .pdr           0x00002ca0       0x20 C:/Program Files/Microchip/MPLAB C32 Suite/bin/../lib/gcc/pic32mx/3.4.4/../../../../pic32mx/lib/size\libc.a(strcpy.o)
 .pdr           0x00002cc0       0x20 C:/Program Files/Microchip/MPLAB C32 Suite/bin/../lib/gcc/pic32mx/3.4.4/../../../../pic32mx/lib/size\libc.a(strlen.o)
 .pdr           0x00002ce0       0x20 C:/Program Files/Microchip/MPLAB C32 Suite/bin/../lib/gcc/pic32mx/3.4.4/../../../../pic32mx/lib/size\libc.a(general-exception.o)
 .pdr           0x00002d00       0x20 C:/Program Files/Microchip/MPLAB C32 Suite/bin/../lib/gcc/pic32mx/3.4.4/../../../../pic32mx/lib/size\libc.a(strcat.o)
 .pdr           0x00002d20       0x20 C:/Program Files/Microchip/MPLAB C32 Suite/bin/../lib/gcc/pic32mx/3.4.4/../../../../pic32mx/lib/size\libc.a(strncmp.o)
 .pdr           0x00002d40       0x20 C:/Program Files/Microchip/MPLAB C32 Suite/bin/../lib/gcc/pic32mx/3.4.4/../../../../pic32mx/lib/size\libc.a(strchr.o)
 .pdr           0x00002d60       0x20 C:/Program Files/Microchip/MPLAB C32 Suite/bin/../lib/gcc/pic32mx/3.4.4/../../../../pic32mx/lib/size\libc.a(strstr.o)
 .pdr           0x00002d80       0x20 C:/Program Files/Microchip/MPLAB C32 Suite/bin/../lib/gcc/pic32mx/3.4.4/../../../../pic32mx/lib/size\libc.a(exit.o)
 .pdr           0x00002da0       0x60 C:/Program Files/Microchip/MPLAB C32 Suite/bin/../lib/gcc/pic32mx/3.4.4/../../../../pic32mx/lib/size\libc.a(rand.o)
 .pdr           0x00002e00       0x20 C:/Program Files/Microchip/MPLAB C32 Suite/bin/../lib/gcc/pic32mx/3.4.4/../../../../pic32mx/lib/size\libc.a(atol.o)
 .pdr           0x00002e20       0x20 C:/Program Files/Microchip/MPLAB C32 Suite/bin/../lib/gcc/pic32mx/3.4.4/../../../../pic32mx/lib/size\libc.a(atoi.o)
 .pdr           0x00002e40       0x20 C:/Program Files/Microchip/MPLAB C32 Suite/bin/../lib/gcc/pic32mx/3.4.4/../../../../pic32mx/lib/size\libc.a(strtol.o)
 .pdr           0x00002e60       0xa0 C:/Program Files/Microchip/MPLAB C32 Suite/bin/../lib/gcc/pic32mx/3.4.4/../../../../pic32mx/lib/size\libc.a(_iobfuncs.o)
 .pdr           0x00002f00      0x2c0 C:/Program Files/Microchip/MPLAB C32 Suite/bin/../lib/gcc/pic32mx/3.4.4/../../../../pic32mx/lib/size\libc.a(stubs.o)
 .pdr           0x000031c0       0x20 C:/Program Files/Microchip/MPLAB C32 Suite/bin/../lib/gcc/pic32mx/3.4.4/../../../../pic32mx/lib/size\libc.a(default-bootstrap-exception-handler.o)
 .pdr           0x000031e0       0x20 C:/Program Files/Microchip/MPLAB C32 Suite/bin/../lib/gcc/pic32mx/3.4.4/../../../../pic32mx/lib/size\libc.a(default-on-reset.o)
 .pdr           0x00003200       0x20 C:/Program Files/Microchip/MPLAB C32 Suite/bin/../lib/gcc/pic32mx/3.4.4/../../../../pic32mx/lib/size\libc.a(default-on-bootstrap.o)
 .pdr           0x00003220       0x20 C:/Program Files/Microchip/MPLAB C32 Suite/bin/../lib/gcc/pic32mx/3.4.4/../../../../pic32mx/lib/size\libc.a(default-nmi-handler.o)
 .pdr           0x00003240       0x20 C:/Program Files/Microchip/MPLAB C32 Suite/bin/../lib/gcc/pic32mx/3.4.4/../../../../pic32mx/lib/size\libc.a(_mon_getc.o)
 .pdr           0x00003260       0x20 C:/Program Files/Microchip/MPLAB C32 Suite/bin/../lib/gcc/pic32mx/3.4.4/../../../../pic32mx/lib/size\libc.a(_mon_write.o)
 .pdr           0x00003280       0x20 C:/Program Files/Microchip/MPLAB C32 Suite/bin/../lib/gcc/pic32mx/3.4.4/../../../../pic32mx/lib/size\libc.a(_exit.o)
 .pdr           0x000032a0       0x20 C:/Program Files/Microchip/MPLAB C32 Suite/bin/../lib/gcc/pic32mx/3.4.4/../../../../pic32mx/lib/size\libc.a(_mon_putc.o)
 .pdr           0x000032c0       0x20 C:/Program Files/Microchip/MPLAB C32 Suite/bin/../lib/gcc/pic32mx/3.4.4/../../../../pic32mx/lib/size\libmchp_peripheral.a(int_disable_interrupts_lib.o)
 .pdr           0x000032e0       0x20 C:/Program Files/Microchip/MPLAB C32 Suite/bin/../lib/gcc/pic32mx/3.4.4/../../../../pic32mx/lib/size\libmchp_peripheral.a(int_enable_mv_int_lib.o)
 .pdr           0x00003300       0x20 C:/Program Files/Microchip/MPLAB C32 Suite/bin/../lib/gcc/pic32mx/3.4.4/../../../../pic32mx/lib/size\libmchp_peripheral.a(int_restore_interrupts_lib.o)
 .pdr           0x00003320       0x40 C:/Program Files/Microchip/MPLAB C32 Suite/bin/../lib/gcc/pic32mx/3.4.4/../../../../pic32mx/lib/size\libmchp_peripheral.a(puts_uartx_lib.o)
 .pdr           0x00003360       0x20 C:/Program Files/Microchip/MPLAB C32 Suite/bin/../lib/gcc/pic32mx/3.4.4/../../../../pic32mx/lib/size\libmchp_peripheral.a(soft_reset_lib.o)
 .pdr           0x00003380       0x40 C:/Program Files/Microchip/MPLAB C32 Suite/bin/../lib/gcc/pic32mx/3.4.4/../../../../pic32mx/lib/size\libmchp_peripheral.a(pcache.o)
 .pdr           0x000033c0       0x20 C:/Program Files/Microchip/MPLAB C32 Suite/bin/../lib/gcc/pic32mx/3.4.4/../../../../pic32mx/lib/size\libmchp_peripheral.a(int_enable_interrupts_lib.o)

.reginfo        0x00000000       0x18
 *(.reginfo)
 .reginfo       0x00000000       0x18 C:/Program Files/Microchip/MPLAB C32 Suite/bin/../lib/gcc/pic32mx/3.4.4/../../../../pic32mx/lib/size/crt0.o

.stab
 *(.stab)

.stabstr
 *(.stabstr)

.stab.excl
 *(.stab.excl)

.stab.exclstr
 *(.stab.exclstr)

.stab.index
 *(.stab.index)

.stab.indexstr
 *(.stab.indexstr)

.comment        0x00000000     0x1fdd
 *(.comment)
 .comment       0x00000000       0x4d Objects - TCPIP Demo App-C32\MainDemo.o
 .comment       0x0000004d       0x4d Objects - TCPIP Demo App-C32\CustomHTTPApp.o
 .comment       0x0000009a       0x4d ..\Microchip\TCPIP Stack\Objects - TCPIP Demo App-C32\UDPPerformanceTest.o
 .comment       0x000000e7       0x4d ..\Microchip\TCPIP Stack\Objects - TCPIP Demo App-C32\Announce.o
 .comment       0x00000134       0x4d ..\Microchip\TCPIP Stack\Objects - TCPIP Demo App-C32\ARP.o
 .comment       0x00000181       0x4d ..\Microchip\TCPIP Stack\Objects - TCPIP Demo App-C32\Delay.o
 .comment       0x000001ce       0x4d ..\Microchip\TCPIP Stack\Objects - TCPIP Demo App-C32\DHCP.o
 .comment       0x0000021b       0x4d ..\Microchip\TCPIP Stack\Objects - TCPIP Demo App-C32\DHCPs.o
 .comment       0x00000268       0x4d ..\Microchip\TCPIP Stack\Objects - TCPIP Demo App-C32\DNS.o
 .comment       0x000002b5       0x4d ..\Microchip\TCPIP Stack\Objects - TCPIP Demo App-C32\DynDNS.o
 .comment       0x00000302       0x4d ..\Microchip\TCPIP Stack\Objects - TCPIP Demo App-C32\ENC28J60.o
 .comment       0x0000034f       0x4d ..\Microchip\TCPIP Stack\Objects - TCPIP Demo App-C32\FTP.o
 .comment       0x0000039c       0x4d ..\Microchip\TCPIP Stack\Objects - TCPIP Demo App-C32\Hashes.o
 .comment       0x000003e9       0x4d ..\Microchip\TCPIP Stack\Objects - TCPIP Demo App-C32\Helpers.o
 .comment       0x00000436       0x4d ..\Microchip\TCPIP Stack\Objects - TCPIP Demo App-C32\HTTP2.o
 .comment       0x00000483       0x4d ..\Microchip\TCPIP Stack\Objects - TCPIP Demo App-C32\HTTP.o
 .comment       0x000004d0       0x4d ..\Microchip\TCPIP Stack\Objects - TCPIP Demo App-C32\ICMP.o
 .comment       0x0000051d       0x4d ..\Microchip\TCPIP Stack\Objects - TCPIP Demo App-C32\IP.o
 .comment       0x0000056a       0x4d ..\Microchip\TCPIP Stack\Objects - TCPIP Demo App-C32\LCDBlocking.o
 .comment       0x000005b7       0x4d ..\Microchip\TCPIP Stack\Objects - TCPIP Demo App-C32\MPFS2.o
 .comment       0x00000604       0x4d ..\Microchip\TCPIP Stack\Objects - TCPIP Demo App-C32\MPFS.o
 .comment       0x00000651       0x4d ..\Microchip\TCPIP Stack\Objects - TCPIP Demo App-C32\NBNS.o
 .comment       0x0000069e       0x4d ..\Microchip\TCPIP Stack\Objects - TCPIP Demo App-C32\Reboot.o
 .comment       0x000006eb       0x4d ..\Microchip\TCPIP Stack\Objects - TCPIP Demo App-C32\SMTP.o
 .comment       0x00000738       0x4d ..\Microchip\TCPIP Stack\Objects - TCPIP Demo App-C32\SNMP.o
 .comment       0x00000785       0x4d ..\Microchip\TCPIP Stack\Objects - TCPIP Demo App-C32\SNTP.o
 .comment       0x000007d2       0x4d ..\Microchip\TCPIP Stack\Objects - TCPIP Demo App-C32\SPIEEPROM.o
 .comment       0x0000081f       0x4d ..\Microchip\TCPIP Stack\Objects - TCPIP Demo App-C32\SPIFlash.o
 .comment       0x0000086c       0x4d ..\Microchip\TCPIP Stack\Objects - TCPIP Demo App-C32\SPIRAM.o
 .comment       0x000008b9       0x4d ..\Microchip\TCPIP Stack\Objects - TCPIP Demo App-C32\StackTsk.o
 .comment       0x00000906       0x4d ..\Microchip\TCPIP Stack\Objects - TCPIP Demo App-C32\TCP.o
 .comment       0x00000953       0x4d ..\Microchip\TCPIP Stack\Objects - TCPIP Demo App-C32\TCPPerformanceTest.o
 .comment       0x000009a0       0x4d ..\Microchip\TCPIP Stack\Objects - TCPIP Demo App-C32\Telnet.o
 .comment       0x000009ed       0x4d ..\Microchip\TCPIP Stack\Objects - TCPIP Demo App-C32\TFTPc.o
 .comment       0x00000a3a       0x4d ..\Microchip\TCPIP Stack\Objects - TCPIP Demo App-C32\Tick.o
 .comment       0x00000a87       0x4d ..\Microchip\TCPIP Stack\Objects - TCPIP Demo App-C32\UART2TCPBridge.o
 .comment       0x00000ad4       0x4d ..\Microchip\TCPIP Stack\Objects - TCPIP Demo App-C32\UART.o
 .comment       0x00000b21       0x4d ..\Microchip\TCPIP Stack\Objects - TCPIP Demo App-C32\UDP.o
 .comment       0x00000b6e       0x4d Objects - TCPIP Demo App-C32\CustomSNMPApp.o
 .comment       0x00000bbb       0x4d Objects - TCPIP Demo App-C32\UARTConfig.o
 .comment       0x00000c08       0x4d Objects - TCPIP Demo App-C32\GenericTCPClient.o
 .comment       0x00000c55       0x4d Objects - TCPIP Demo App-C32\GenericTCPServer.o
 .comment       0x00000ca2       0x4d Objects - TCPIP Demo App-C32\LegacyHTTPApp.o
 .comment       0x00000cef       0x4d Objects - TCPIP Demo App-C32\PingDemo.o
 .comment       0x00000d3c       0x4d Objects - TCPIP Demo App-C32\SMTPDemo.o
 .comment       0x00000d89       0x4d ..\Microchip\TCPIP Stack\Objects - TCPIP Demo App-C32\BerkeleyAPI.o
 .comment       0x00000dd6       0x4d Objects - TCPIP Demo App-C32\BerkeleyUDPClientDemo.o
 .comment       0x00000e23       0x4d Objects - TCPIP Demo App-C32\BerkeleyTCPClientDemo.o
 .comment       0x00000e70       0x4d Objects - TCPIP Demo App-C32\BerkeleyTCPServerDemo.o
 .comment       0x00000ebd       0x4d ..\Microchip\TCPIP Stack\Objects - TCPIP Demo App-C32\ENCX24J600.o
 .comment       0x00000f0a       0x4d Objects - TCPIP Demo App-C32\MPFSImg2.o
 .comment       0x00000f57       0x4d ..\Microchip\TCPIP Stack\Objects - TCPIP Demo App-C32\Random.o
 .comment       0x00000fa4       0x4d ..\Microchip\TCPIP Stack\Objects - TCPIP Demo App-C32\RSA.o
 .comment       0x00000ff1       0x4d ..\Microchip\TCPIP Stack\Objects - TCPIP Demo App-C32\SSL.o
 .comment       0x0000103e       0x4d ..\Microchip\TCPIP Stack\Objects - TCPIP Demo App-C32\ARCFOUR.o
 .comment       0x0000108b       0x4d ..\Microchip\TCPIP Stack\Objects - TCPIP Demo App-C32\BigInt.o
 .comment       0x000010d8       0x4d Objects - TCPIP Demo App-C32\CustomSSLCert.o
 .comment       0x00001125       0x4d C:/Program Files/Microchip/MPLAB C32 Suite/bin/../lib/gcc/pic32mx/3.4.4/size\libgcc.a(_udivdi3.o)
 .comment       0x00001172       0x56 C:/Program Files/Microchip/MPLAB C32 Suite/bin/../lib/gcc/pic32mx/3.4.4/../../../../pic32mx/lib/size\libc.a(memcmp.o)
 .comment       0x000011c8       0x56 C:/Program Files/Microchip/MPLAB C32 Suite/bin/../lib/gcc/pic32mx/3.4.4/../../../../pic32mx/lib/size\libc.a(memset.o)
 .comment       0x0000121e       0x56 C:/Program Files/Microchip/MPLAB C32 Suite/bin/../lib/gcc/pic32mx/3.4.4/../../../../pic32mx/lib/size\libc.a(strcmp.o)
 .comment       0x00001274       0x56 C:/Program Files/Microchip/MPLAB C32 Suite/bin/../lib/gcc/pic32mx/3.4.4/../../../../pic32mx/lib/size\libc.a(strcpy.o)
 .comment       0x000012ca       0x56 C:/Program Files/Microchip/MPLAB C32 Suite/bin/../lib/gcc/pic32mx/3.4.4/../../../../pic32mx/lib/size\libc.a(strlen.o)
 .comment       0x00001320       0x9c C:/Program Files/Microchip/MPLAB C32 Suite/bin/../lib/gcc/pic32mx/3.4.4/../../../../pic32mx/lib/size\libc.a(strcat.o)
 .comment       0x000013bc       0x9d C:/Program Files/Microchip/MPLAB C32 Suite/bin/../lib/gcc/pic32mx/3.4.4/../../../../pic32mx/lib/size\libc.a(strncmp.o)
 .comment       0x00001459       0x9c C:/Program Files/Microchip/MPLAB C32 Suite/bin/../lib/gcc/pic32mx/3.4.4/../../../../pic32mx/lib/size\libc.a(strchr.o)
 .comment       0x000014f5       0x9c C:/Program Files/Microchip/MPLAB C32 Suite/bin/../lib/gcc/pic32mx/3.4.4/../../../../pic32mx/lib/size\libc.a(strstr.o)
 .comment       0x00001591       0x9a C:/Program Files/Microchip/MPLAB C32 Suite/bin/../lib/gcc/pic32mx/3.4.4/../../../../pic32mx/lib/size\libc.a(exit.o)
 .comment       0x0000162b       0x9a C:/Program Files/Microchip/MPLAB C32 Suite/bin/../lib/gcc/pic32mx/3.4.4/../../../../pic32mx/lib/size\libc.a(rand.o)
 .comment       0x000016c5       0x9a C:/Program Files/Microchip/MPLAB C32 Suite/bin/../lib/gcc/pic32mx/3.4.4/../../../../pic32mx/lib/size\libc.a(atol.o)
 .comment       0x0000175f       0x9a C:/Program Files/Microchip/MPLAB C32 Suite/bin/../lib/gcc/pic32mx/3.4.4/../../../../pic32mx/lib/size\libc.a(atoi.o)
 .comment       0x000017f9       0x9c C:/Program Files/Microchip/MPLAB C32 Suite/bin/../lib/gcc/pic32mx/3.4.4/../../../../pic32mx/lib/size\libc.a(strtol.o)
 .comment       0x00001895       0xa0 C:/Program Files/Microchip/MPLAB C32 Suite/bin/../lib/gcc/pic32mx/3.4.4/../../../../pic32mx/lib/size\libc.a(_iobdata.o)
 .comment       0x00001935       0xa1 C:/Program Files/Microchip/MPLAB C32 Suite/bin/../lib/gcc/pic32mx/3.4.4/../../../../pic32mx/lib/size\libc.a(_iobfuncs.o)
 .comment       0x000019d6       0x9b C:/Program Files/Microchip/MPLAB C32 Suite/bin/../lib/gcc/pic32mx/3.4.4/../../../../pic32mx/lib/size\libc.a(stubs.o)
 .comment       0x00001a71       0x4d C:/Program Files/Microchip/MPLAB C32 Suite/bin/../lib/gcc/pic32mx/3.4.4/../../../../pic32mx/lib/size\libc.a(default-bootstrap-exception-handler.o)
 .comment       0x00001abe       0x4d C:/Program Files/Microchip/MPLAB C32 Suite/bin/../lib/gcc/pic32mx/3.4.4/../../../../pic32mx/lib/size\libc.a(default-on-reset.o)
 .comment       0x00001b0b       0x4d C:/Program Files/Microchip/MPLAB C32 Suite/bin/../lib/gcc/pic32mx/3.4.4/../../../../pic32mx/lib/size\libc.a(default-on-bootstrap.o)
 .comment       0x00001b58       0x4d C:/Program Files/Microchip/MPLAB C32 Suite/bin/../lib/gcc/pic32mx/3.4.4/../../../../pic32mx/lib/size\libc.a(_mon_getc.o)
 .comment       0x00001ba5       0x4d C:/Program Files/Microchip/MPLAB C32 Suite/bin/../lib/gcc/pic32mx/3.4.4/../../../../pic32mx/lib/size\libc.a(_mon_write.o)
 .comment       0x00001bf2       0x4d C:/Program Files/Microchip/MPLAB C32 Suite/bin/../lib/gcc/pic32mx/3.4.4/../../../../pic32mx/lib/size\libc.a(_exit.o)
 .comment       0x00001c3f       0x9b C:/Program Files/Microchip/MPLAB C32 Suite/bin/../lib/gcc/pic32mx/3.4.4/../../../../pic32mx/lib/size\libc.a(ctype.o)
 .comment       0x00001cda       0x9b C:/Program Files/Microchip/MPLAB C32 Suite/bin/../lib/gcc/pic32mx/3.4.4/../../../../pic32mx/lib/size\libc.a(errno.o)
 .comment       0x00001d75       0x4d C:/Program Files/Microchip/MPLAB C32 Suite/bin/../lib/gcc/pic32mx/3.4.4/../../../../pic32mx/lib/size\libc.a(_mon_putc.o)
 .comment       0x00001dc2       0x4d C:/Program Files/Microchip/MPLAB C32 Suite/bin/../lib/gcc/pic32mx/3.4.4/../../../../pic32mx/lib/size\libmchp_peripheral.a(int_disable_interrupts_lib.o)
 .comment       0x00001e0f       0x4d C:/Program Files/Microchip/MPLAB C32 Suite/bin/../lib/gcc/pic32mx/3.4.4/../../../../pic32mx/lib/size\libmchp_peripheral.a(int_enable_mv_int_lib.o)
 .comment       0x00001e5c       0x4d C:/Program Files/Microchip/MPLAB C32 Suite/bin/../lib/gcc/pic32mx/3.4.4/../../../../pic32mx/lib/size\libmchp_peripheral.a(int_restore_interrupts_lib.o)
 .comment       0x00001ea9       0x4d C:/Program Files/Microchip/MPLAB C32 Suite/bin/../lib/gcc/pic32mx/3.4.4/../../../../pic32mx/lib/size\libmchp_peripheral.a(puts_uartx_lib.o)
 .comment       0x00001ef6       0x4d C:/Program Files/Microchip/MPLAB C32 Suite/bin/../lib/gcc/pic32mx/3.4.4/../../../../pic32mx/lib/size\libmchp_peripheral.a(soft_reset_lib.o)
 .comment       0x00001f43       0x4d C:/Program Files/Microchip/MPLAB C32 Suite/bin/../lib/gcc/pic32mx/3.4.4/../../../../pic32mx/lib/size\libmchp_peripheral.a(pcache.o)
 .comment       0x00001f90       0x4d C:/Program Files/Microchip/MPLAB C32 Suite/bin/../lib/gcc/pic32mx/3.4.4/../../../../pic32mx/lib/size\libmchp_peripheral.a(int_enable_interrupts_lib.o)

.debug
 *(.debug)

.line
 *(.line)

.debug_srcinfo
 *(.debug_srcinfo)

.debug_sfnames
 *(.debug_sfnames)

.debug_aranges  0x00000000      0x520
 *(.debug_aranges)
 .debug_aranges
                0x00000000       0x20 Objects - TCPIP Demo App-C32\MainDemo.o
 .debug_aranges
                0x00000020       0x20 Objects - TCPIP Demo App-C32\CustomHTTPApp.o
 .debug_aranges
                0x00000040       0x20 ..\Microchip\TCPIP Stack\Objects - TCPIP Demo App-C32\Announce.o
 .debug_aranges
                0x00000060       0x20 ..\Microchip\TCPIP Stack\Objects - TCPIP Demo App-C32\ARP.o
 .debug_aranges
                0x00000080       0x20 ..\Microchip\TCPIP Stack\Objects - TCPIP Demo App-C32\Delay.o
 .debug_aranges
                0x000000a0       0x20 ..\Microchip\TCPIP Stack\Objects - TCPIP Demo App-C32\DHCP.o
 .debug_aranges
                0x000000c0       0x20 ..\Microchip\TCPIP Stack\Objects - TCPIP Demo App-C32\DHCPs.o
 .debug_aranges
                0x000000e0       0x20 ..\Microchip\TCPIP Stack\Objects - TCPIP Demo App-C32\DNS.o
 .debug_aranges
                0x00000100       0x20 ..\Microchip\TCPIP Stack\Objects - TCPIP Demo App-C32\DynDNS.o
 .debug_aranges
                0x00000120       0x20 ..\Microchip\TCPIP Stack\Objects - TCPIP Demo App-C32\ENC28J60.o
 .debug_aranges
                0x00000140       0x20 ..\Microchip\TCPIP Stack\Objects - TCPIP Demo App-C32\Hashes.o
 .debug_aranges
                0x00000160       0x20 ..\Microchip\TCPIP Stack\Objects - TCPIP Demo App-C32\Helpers.o
 .debug_aranges
                0x00000180       0x20 ..\Microchip\TCPIP Stack\Objects - TCPIP Demo App-C32\HTTP2.o
 .debug_aranges
                0x000001a0       0x20 ..\Microchip\TCPIP Stack\Objects - TCPIP Demo App-C32\ICMP.o
 .debug_aranges
                0x000001c0       0x20 ..\Microchip\TCPIP Stack\Objects - TCPIP Demo App-C32\IP.o
 .debug_aranges
                0x000001e0       0x20 ..\Microchip\TCPIP Stack\Objects - TCPIP Demo App-C32\LCDBlocking.o
 .debug_aranges
                0x00000200       0x20 ..\Microchip\TCPIP Stack\Objects - TCPIP Demo App-C32\MPFS2.o
 .debug_aranges
                0x00000220       0x20 ..\Microchip\TCPIP Stack\Objects - TCPIP Demo App-C32\NBNS.o
 .debug_aranges
                0x00000240       0x20 ..\Microchip\TCPIP Stack\Objects - TCPIP Demo App-C32\Reboot.o
 .debug_aranges
                0x00000260       0x20 ..\Microchip\TCPIP Stack\Objects - TCPIP Demo App-C32\SMTP.o
 .debug_aranges
                0x00000280       0x20 ..\Microchip\TCPIP Stack\Objects - TCPIP Demo App-C32\SNMP.o
 .debug_aranges
                0x000002a0       0x20 ..\Microchip\TCPIP Stack\Objects - TCPIP Demo App-C32\SNTP.o
 .debug_aranges
                0x000002c0       0x20 ..\Microchip\TCPIP Stack\Objects - TCPIP Demo App-C32\SPIEEPROM.o
 .debug_aranges
                0x000002e0       0x20 ..\Microchip\TCPIP Stack\Objects - TCPIP Demo App-C32\StackTsk.o
 .debug_aranges
                0x00000300       0x20 ..\Microchip\TCPIP Stack\Objects - TCPIP Demo App-C32\TCP.o
 .debug_aranges
                0x00000320       0x20 ..\Microchip\TCPIP Stack\Objects - TCPIP Demo App-C32\TCPPerformanceTest.o
 .debug_aranges
                0x00000340       0x20 ..\Microchip\TCPIP Stack\Objects - TCPIP Demo App-C32\Telnet.o
 .debug_aranges
                0x00000360       0x20 ..\Microchip\TCPIP Stack\Objects - TCPIP Demo App-C32\Tick.o
 .debug_aranges
                0x00000380       0x20 ..\Microchip\TCPIP Stack\Objects - TCPIP Demo App-C32\UART2TCPBridge.o
 .debug_aranges
                0x000003a0       0x20 ..\Microchip\TCPIP Stack\Objects - TCPIP Demo App-C32\UART.o
 .debug_aranges
                0x000003c0       0x20 ..\Microchip\TCPIP Stack\Objects - TCPIP Demo App-C32\UDP.o
 .debug_aranges
                0x000003e0       0x20 Objects - TCPIP Demo App-C32\CustomSNMPApp.o
 .debug_aranges
                0x00000400       0x20 Objects - TCPIP Demo App-C32\UARTConfig.o
 .debug_aranges
                0x00000420       0x20 Objects - TCPIP Demo App-C32\GenericTCPClient.o
 .debug_aranges
                0x00000440       0x20 Objects - TCPIP Demo App-C32\GenericTCPServer.o
 .debug_aranges
                0x00000460       0x20 Objects - TCPIP Demo App-C32\PingDemo.o
 .debug_aranges
                0x00000480       0x20 Objects - TCPIP Demo App-C32\SMTPDemo.o
 .debug_aranges
                0x000004a0       0x20 ..\Microchip\TCPIP Stack\Objects - TCPIP Demo App-C32\BerkeleyAPI.o
 .debug_aranges
                0x000004c0       0x20 Objects - TCPIP Demo App-C32\BerkeleyUDPClientDemo.o
 .debug_aranges
                0x000004e0       0x20 Objects - TCPIP Demo App-C32\BerkeleyTCPClientDemo.o
 .debug_aranges
                0x00000500       0x20 Objects - TCPIP Demo App-C32\BerkeleyTCPServerDemo.o

.debug_pubnames
                0x00000000     0x173b
 *(.debug_pubnames)
 .debug_pubnames
                0x00000000       0x9e Objects - TCPIP Demo App-C32\MainDemo.o
 .debug_pubnames
                0x0000009e      0x3a2 Objects - TCPIP Demo App-C32\CustomHTTPApp.o
 .debug_pubnames
                0x00000440       0x33 ..\Microchip\TCPIP Stack\Objects - TCPIP Demo App-C32\Announce.o
 .debug_pubnames
                0x00000473       0x4e ..\Microchip\TCPIP Stack\Objects - TCPIP Demo App-C32\ARP.o
 .debug_pubnames
                0x000004c1       0x2c ..\Microchip\TCPIP Stack\Objects - TCPIP Demo App-C32\Delay.o
 .debug_pubnames
                0x000004ed       0x7c ..\Microchip\TCPIP Stack\Objects - TCPIP Demo App-C32\DHCP.o
 .debug_pubnames
                0x00000569       0x3c ..\Microchip\TCPIP Stack\Objects - TCPIP Demo App-C32\DHCPs.o
 .debug_pubnames
                0x000005a5       0x55 ..\Microchip\TCPIP Stack\Objects - TCPIP Demo App-C32\DNS.o
 .debug_pubnames
                0x000005fa       0x9f ..\Microchip\TCPIP Stack\Objects - TCPIP Demo App-C32\DynDNS.o
 .debug_pubnames
                0x00000699      0x1b8 ..\Microchip\TCPIP Stack\Objects - TCPIP Demo App-C32\ENC28J60.o
 .debug_pubnames
                0x00000851       0x62 ..\Microchip\TCPIP Stack\Objects - TCPIP Demo App-C32\Hashes.o
 .debug_pubnames
                0x000008b3       0xfe ..\Microchip\TCPIP Stack\Objects - TCPIP Demo App-C32\Helpers.o
 .debug_pubnames
                0x000009b1       0xcf ..\Microchip\TCPIP Stack\Objects - TCPIP Demo App-C32\HTTP2.o
 .debug_pubnames
                0x00000a80       0x7f ..\Microchip\TCPIP Stack\Objects - TCPIP Demo App-C32\ICMP.o
 .debug_pubnames
                0x00000aff       0x44 ..\Microchip\TCPIP Stack\Objects - TCPIP Demo App-C32\IP.o
 .debug_pubnames
                0x00000b43       0x45 ..\Microchip\TCPIP Stack\Objects - TCPIP Demo App-C32\LCDBlocking.o
 .debug_pubnames
                0x00000b88      0x17c ..\Microchip\TCPIP Stack\Objects - TCPIP Demo App-C32\MPFS2.o
 .debug_pubnames
                0x00000d04       0x1f ..\Microchip\TCPIP Stack\Objects - TCPIP Demo App-C32\NBNS.o
 .debug_pubnames
                0x00000d23       0x21 ..\Microchip\TCPIP Stack\Objects - TCPIP Demo App-C32\Reboot.o
 .debug_pubnames
                0x00000d44       0xd2 ..\Microchip\TCPIP Stack\Objects - TCPIP Demo App-C32\SMTP.o
 .debug_pubnames
                0x00000e16       0x7f ..\Microchip\TCPIP Stack\Objects - TCPIP Demo App-C32\SNMP.o
 .debug_pubnames
                0x00000e95       0x37 ..\Microchip\TCPIP Stack\Objects - TCPIP Demo App-C32\SNTP.o
 .debug_pubnames
                0x00000ecc       0xaa ..\Microchip\TCPIP Stack\Objects - TCPIP Demo App-C32\SPIEEPROM.o
 .debug_pubnames
                0x00000f76       0x53 ..\Microchip\TCPIP Stack\Objects - TCPIP Demo App-C32\StackTsk.o
 .debug_pubnames
                0x00000fc9      0x190 ..\Microchip\TCPIP Stack\Objects - TCPIP Demo App-C32\TCP.o
 .debug_pubnames
                0x00001159       0x5b ..\Microchip\TCPIP Stack\Objects - TCPIP Demo App-C32\TCPPerformanceTest.o
 .debug_pubnames
                0x000011b4       0x21 ..\Microchip\TCPIP Stack\Objects - TCPIP Demo App-C32\Telnet.o
 .debug_pubnames
                0x000011d5       0x7e ..\Microchip\TCPIP Stack\Objects - TCPIP Demo App-C32\Tick.o
 .debug_pubnames
                0x00001253       0x76 ..\Microchip\TCPIP Stack\Objects - TCPIP Demo App-C32\UART2TCPBridge.o
 .debug_pubnames
                0x000012c9       0x25 ..\Microchip\TCPIP Stack\Objects - TCPIP Demo App-C32\UART.o
 .debug_pubnames
                0x000012ee      0x143 ..\Microchip\TCPIP Stack\Objects - TCPIP Demo App-C32\UDP.o
 .debug_pubnames
                0x00001431      0x110 Objects - TCPIP Demo App-C32\CustomSNMPApp.o
 .debug_pubnames
                0x00001541       0x23 Objects - TCPIP Demo App-C32\UARTConfig.o
 .debug_pubnames
                0x00001564       0x27 Objects - TCPIP Demo App-C32\GenericTCPClient.o
 .debug_pubnames
                0x0000158b       0x27 Objects - TCPIP Demo App-C32\GenericTCPServer.o
 .debug_pubnames
                0x000015b2       0x1f Objects - TCPIP Demo App-C32\PingDemo.o
 .debug_pubnames
                0x000015d1       0x1f Objects - TCPIP Demo App-C32\SMTPDemo.o
 .debug_pubnames
                0x000015f0       0xa9 ..\Microchip\TCPIP Stack\Objects - TCPIP Demo App-C32\BerkeleyAPI.o
 .debug_pubnames
                0x00001699       0x4a Objects - TCPIP Demo App-C32\BerkeleyUDPClientDemo.o
 .debug_pubnames
                0x000016e3       0x2c Objects - TCPIP Demo App-C32\BerkeleyTCPClientDemo.o
 .debug_pubnames
                0x0000170f       0x2c Objects - TCPIP Demo App-C32\BerkeleyTCPServerDemo.o

.debug_info     0x00000000    0x28997
 *(.debug_info .gnu.linkonce.wi.*)
 .debug_info    0x00000000     0x14d2 Objects - TCPIP Demo App-C32\MainDemo.o
 .debug_info    0x000014d2     0x2012 Objects - TCPIP Demo App-C32\CustomHTTPApp.o
 .debug_info    0x000034e4      0x392 ..\Microchip\TCPIP Stack\Objects - TCPIP Demo App-C32\UDPPerformanceTest.o
 .debug_info    0x00003876      0xc58 ..\Microchip\TCPIP Stack\Objects - TCPIP Demo App-C32\Announce.o
 .debug_info    0x000044ce      0xd4b ..\Microchip\TCPIP Stack\Objects - TCPIP Demo App-C32\ARP.o
 .debug_info    0x00005219      0x418 ..\Microchip\TCPIP Stack\Objects - TCPIP Demo App-C32\Delay.o
 .debug_info    0x00005631     0x10df ..\Microchip\TCPIP Stack\Objects - TCPIP Demo App-C32\DHCP.o
 .debug_info    0x00006710      0xe97 ..\Microchip\TCPIP Stack\Objects - TCPIP Demo App-C32\DHCPs.o
 .debug_info    0x000075a7     0x100b ..\Microchip\TCPIP Stack\Objects - TCPIP Demo App-C32\DNS.o
 .debug_info    0x000085b2     0x110f ..\Microchip\TCPIP Stack\Objects - TCPIP Demo App-C32\DynDNS.o
 .debug_info    0x000096c1     0x2a0d ..\Microchip\TCPIP Stack\Objects - TCPIP Demo App-C32\ENC28J60.o
 .debug_info    0x0000c0ce      0x383 ..\Microchip\TCPIP Stack\Objects - TCPIP Demo App-C32\FTP.o
 .debug_info    0x0000c451      0x766 ..\Microchip\TCPIP Stack\Objects - TCPIP Demo App-C32\Hashes.o
 .debug_info    0x0000cbb7      0xfdf ..\Microchip\TCPIP Stack\Objects - TCPIP Demo App-C32\Helpers.o
 .debug_info    0x0000db96     0x11c8 ..\Microchip\TCPIP Stack\Objects - TCPIP Demo App-C32\HTTP2.o
 .debug_info    0x0000ed5e      0x384 ..\Microchip\TCPIP Stack\Objects - TCPIP Demo App-C32\HTTP.o
 .debug_info    0x0000f0e2      0xced ..\Microchip\TCPIP Stack\Objects - TCPIP Demo App-C32\ICMP.o
 .debug_info    0x0000fdcf      0xd79 ..\Microchip\TCPIP Stack\Objects - TCPIP Demo App-C32\IP.o
 .debug_info    0x00010b48      0x574 ..\Microchip\TCPIP Stack\Objects - TCPIP Demo App-C32\LCDBlocking.o
 .debug_info    0x000110bc      0xbb9 ..\Microchip\TCPIP Stack\Objects - TCPIP Demo App-C32\MPFS2.o
 .debug_info    0x00011c75      0x384 ..\Microchip\TCPIP Stack\Objects - TCPIP Demo App-C32\MPFS.o
 .debug_info    0x00011ff9      0xd8a ..\Microchip\TCPIP Stack\Objects - TCPIP Demo App-C32\NBNS.o
 .debug_info    0x00012d83      0xbc1 ..\Microchip\TCPIP Stack\Objects - TCPIP Demo App-C32\Reboot.o
 .debug_info    0x00013944     0x1635 ..\Microchip\TCPIP Stack\Objects - TCPIP Demo App-C32\SMTP.o
 .debug_info    0x00014f79     0x29ca ..\Microchip\TCPIP Stack\Objects - TCPIP Demo App-C32\SNMP.o
 .debug_info    0x00017943      0xcdc ..\Microchip\TCPIP Stack\Objects - TCPIP Demo App-C32\SNTP.o
 .debug_info    0x0001861f      0x9ae ..\Microchip\TCPIP Stack\Objects - TCPIP Demo App-C32\SPIEEPROM.o
 .debug_info    0x00018fcd      0x388 ..\Microchip\TCPIP Stack\Objects - TCPIP Demo App-C32\SPIFlash.o
 .debug_info    0x00019355      0x386 ..\Microchip\TCPIP Stack\Objects - TCPIP Demo App-C32\SPIRAM.o
 .debug_info    0x000196db      0xcbf ..\Microchip\TCPIP Stack\Objects - TCPIP Demo App-C32\StackTsk.o
 .debug_info    0x0001a39a     0x22c6 ..\Microchip\TCPIP Stack\Objects - TCPIP Demo App-C32\TCP.o
 .debug_info    0x0001c660      0xa6a ..\Microchip\TCPIP Stack\Objects - TCPIP Demo App-C32\TCPPerformanceTest.o
 .debug_info    0x0001d0ca      0x7c0 ..\Microchip\TCPIP Stack\Objects - TCPIP Demo App-C32\Telnet.o
 .debug_info    0x0001d88a      0x385 ..\Microchip\TCPIP Stack\Objects - TCPIP Demo App-C32\TFTPc.o
 .debug_info    0x0001dc0f      0xb12 ..\Microchip\TCPIP Stack\Objects - TCPIP Demo App-C32\Tick.o
 .debug_info    0x0001e721      0x79b ..\Microchip\TCPIP Stack\Objects - TCPIP Demo App-C32\UART2TCPBridge.o
 .debug_info    0x0001eebc      0x449 ..\Microchip\TCPIP Stack\Objects - TCPIP Demo App-C32\UART.o
 .debug_info    0x0001f305     0x1278 ..\Microchip\TCPIP Stack\Objects - TCPIP Demo App-C32\UDP.o
 .debug_info    0x0002057d     0x1257 Objects - TCPIP Demo App-C32\CustomSNMPApp.o
 .debug_info    0x000217d4      0xb7a Objects - TCPIP Demo App-C32\UARTConfig.o
 .debug_info    0x0002234e      0x58f Objects - TCPIP Demo App-C32\GenericTCPClient.o
 .debug_info    0x000228dd      0x4bc Objects - TCPIP Demo App-C32\GenericTCPServer.o
 .debug_info    0x00022d99      0x381 Objects - TCPIP Demo App-C32\LegacyHTTPApp.o
 .debug_info    0x0002311a      0x488 Objects - TCPIP Demo App-C32\PingDemo.o
 .debug_info    0x000235a2      0x838 Objects - TCPIP Demo App-C32\SMTPDemo.o
 .debug_info    0x00023dda     0x14b8 ..\Microchip\TCPIP Stack\Objects - TCPIP Demo App-C32\BerkeleyAPI.o
 .debug_info    0x00025292      0xdbc Objects - TCPIP Demo App-C32\BerkeleyUDPClientDemo.o
 .debug_info    0x0002604e      0x6c9 Objects - TCPIP Demo App-C32\BerkeleyTCPClientDemo.o
 .debug_info    0x00026717      0x660 Objects - TCPIP Demo App-C32\BerkeleyTCPServerDemo.o
 .debug_info    0x00026d77      0x38a ..\Microchip\TCPIP Stack\Objects - TCPIP Demo App-C32\ENCX24J600.o
 .debug_info    0x00027101      0x37c Objects - TCPIP Demo App-C32\MPFSImg2.o
 .debug_info    0x0002747d      0x386 ..\Microchip\TCPIP Stack\Objects - TCPIP Demo App-C32\Random.o
 .debug_info    0x00027803      0x383 ..\Microchip\TCPIP Stack\Objects - TCPIP Demo App-C32\RSA.o
 .debug_info    0x00027b86      0x383 ..\Microchip\TCPIP Stack\Objects - TCPIP Demo App-C32\SSL.o
 .debug_info    0x00027f09      0x387 ..\Microchip\TCPIP Stack\Objects - TCPIP Demo App-C32\ARCFOUR.o
 .debug_info    0x00028290      0x386 ..\Microchip\TCPIP Stack\Objects - TCPIP Demo App-C32\BigInt.o
 .debug_info    0x00028616      0x381 Objects - TCPIP Demo App-C32\CustomSSLCert.o

.debug_abbrev   0x00000000     0x536c
 *(.debug_abbrev)
 .debug_abbrev  0x00000000      0x2f3 Objects - TCPIP Demo App-C32\MainDemo.o
 .debug_abbrev  0x000002f3      0x287 Objects - TCPIP Demo App-C32\CustomHTTPApp.o
 .debug_abbrev  0x0000057a       0xab ..\Microchip\TCPIP Stack\Objects - TCPIP Demo App-C32\UDPPerformanceTest.o
 .debug_abbrev  0x00000625      0x184 ..\Microchip\TCPIP Stack\Objects - TCPIP Demo App-C32\Announce.o
 .debug_abbrev  0x000007a9      0x23a ..\Microchip\TCPIP Stack\Objects - TCPIP Demo App-C32\ARP.o
 .debug_abbrev  0x000009e3       0xe0 ..\Microchip\TCPIP Stack\Objects - TCPIP Demo App-C32\Delay.o
 .debug_abbrev  0x00000ac3      0x1e1 ..\Microchip\TCPIP Stack\Objects - TCPIP Demo App-C32\DHCP.o
 .debug_abbrev  0x00000ca4      0x1ba ..\Microchip\TCPIP Stack\Objects - TCPIP Demo App-C32\DHCPs.o
 .debug_abbrev  0x00000e5e      0x200 ..\Microchip\TCPIP Stack\Objects - TCPIP Demo App-C32\DNS.o
 .debug_abbrev  0x0000105e      0x21b ..\Microchip\TCPIP Stack\Objects - TCPIP Demo App-C32\DynDNS.o
 .debug_abbrev  0x00001279      0x2ce ..\Microchip\TCPIP Stack\Objects - TCPIP Demo App-C32\ENC28J60.o
 .debug_abbrev  0x00001547       0xab ..\Microchip\TCPIP Stack\Objects - TCPIP Demo App-C32\FTP.o
 .debug_abbrev  0x000015f2      0x1ad ..\Microchip\TCPIP Stack\Objects - TCPIP Demo App-C32\Hashes.o
 .debug_abbrev  0x0000179f      0x1c0 ..\Microchip\TCPIP Stack\Objects - TCPIP Demo App-C32\Helpers.o
 .debug_abbrev  0x0000195f      0x241 ..\Microchip\TCPIP Stack\Objects - TCPIP Demo App-C32\HTTP2.o
 .debug_abbrev  0x00001ba0       0xab ..\Microchip\TCPIP Stack\Objects - TCPIP Demo App-C32\HTTP.o
 .debug_abbrev  0x00001c4b      0x1e4 ..\Microchip\TCPIP Stack\Objects - TCPIP Demo App-C32\ICMP.o
 .debug_abbrev  0x00001e2f      0x1bb ..\Microchip\TCPIP Stack\Objects - TCPIP Demo App-C32\IP.o
 .debug_abbrev  0x00001fea      0x153 ..\Microchip\TCPIP Stack\Objects - TCPIP Demo App-C32\LCDBlocking.o
 .debug_abbrev  0x0000213d      0x209 ..\Microchip\TCPIP Stack\Objects - TCPIP Demo App-C32\MPFS2.o
 .debug_abbrev  0x00002346       0xab ..\Microchip\TCPIP Stack\Objects - TCPIP Demo App-C32\MPFS.o
 .debug_abbrev  0x000023f1      0x1a2 ..\Microchip\TCPIP Stack\Objects - TCPIP Demo App-C32\NBNS.o
 .debug_abbrev  0x00002593      0x13f ..\Microchip\TCPIP Stack\Objects - TCPIP Demo App-C32\Reboot.o
 .debug_abbrev  0x000026d2      0x2a5 ..\Microchip\TCPIP Stack\Objects - TCPIP Demo App-C32\SMTP.o
 .debug_abbrev  0x00002977      0x290 ..\Microchip\TCPIP Stack\Objects - TCPIP Demo App-C32\SNMP.o
 .debug_abbrev  0x00002c07      0x17d ..\Microchip\TCPIP Stack\Objects - TCPIP Demo App-C32\SNTP.o
 .debug_abbrev  0x00002d84      0x231 ..\Microchip\TCPIP Stack\Objects - TCPIP Demo App-C32\SPIEEPROM.o
 .debug_abbrev  0x00002fb5       0xab ..\Microchip\TCPIP Stack\Objects - TCPIP Demo App-C32\SPIFlash.o
 .debug_abbrev  0x00003060       0xab ..\Microchip\TCPIP Stack\Objects - TCPIP Demo App-C32\SPIRAM.o
 .debug_abbrev  0x0000310b      0x192 ..\Microchip\TCPIP Stack\Objects - TCPIP Demo App-C32\StackTsk.o
 .debug_abbrev  0x0000329d      0x269 ..\Microchip\TCPIP Stack\Objects - TCPIP Demo App-C32\TCP.o
 .debug_abbrev  0x00003506      0x189 ..\Microchip\TCPIP Stack\Objects - TCPIP Demo App-C32\TCPPerformanceTest.o
 .debug_abbrev  0x0000368f      0x127 ..\Microchip\TCPIP Stack\Objects - TCPIP Demo App-C32\Telnet.o
 .debug_abbrev  0x000037b6       0xab ..\Microchip\TCPIP Stack\Objects - TCPIP Demo App-C32\TFTPc.o
 .debug_abbrev  0x00003861      0x1c8 ..\Microchip\TCPIP Stack\Objects - TCPIP Demo App-C32\Tick.o
 .debug_abbrev  0x00003a29      0x154 ..\Microchip\TCPIP Stack\Objects - TCPIP Demo App-C32\UART2TCPBridge.o
 .debug_abbrev  0x00003b7d       0xeb ..\Microchip\TCPIP Stack\Objects - TCPIP Demo App-C32\UART.o
 .debug_abbrev  0x00003c68      0x25e ..\Microchip\TCPIP Stack\Objects - TCPIP Demo App-C32\UDP.o
 .debug_abbrev  0x00003ec6      0x277 Objects - TCPIP Demo App-C32\CustomSNMPApp.o
 .debug_abbrev  0x0000413d      0x16d Objects - TCPIP Demo App-C32\UARTConfig.o
 .debug_abbrev  0x000042aa      0x102 Objects - TCPIP Demo App-C32\GenericTCPClient.o
 .debug_abbrev  0x000043ac       0xfb Objects - TCPIP Demo App-C32\GenericTCPServer.o
 .debug_abbrev  0x000044a7       0xab Objects - TCPIP Demo App-C32\LegacyHTTPApp.o
 .debug_abbrev  0x00004552       0xf9 Objects - TCPIP Demo App-C32\PingDemo.o
 .debug_abbrev  0x0000464b      0x181 Objects - TCPIP Demo App-C32\SMTPDemo.o
 .debug_abbrev  0x000047cc      0x237 ..\Microchip\TCPIP Stack\Objects - TCPIP Demo App-C32\BerkeleyAPI.o
 .debug_abbrev  0x00004a03      0x18a Objects - TCPIP Demo App-C32\BerkeleyUDPClientDemo.o
 .debug_abbrev  0x00004b8d      0x147 Objects - TCPIP Demo App-C32\BerkeleyTCPClientDemo.o
 .debug_abbrev  0x00004cd4      0x140 Objects - TCPIP Demo App-C32\BerkeleyTCPServerDemo.o
 .debug_abbrev  0x00004e14       0xab ..\Microchip\TCPIP Stack\Objects - TCPIP Demo App-C32\ENCX24J600.o
 .debug_abbrev  0x00004ebf       0xab Objects - TCPIP Demo App-C32\MPFSImg2.o
 .debug_abbrev  0x00004f6a       0xab ..\Microchip\TCPIP Stack\Objects - TCPIP Demo App-C32\Random.o
 .debug_abbrev  0x00005015       0xab ..\Microchip\TCPIP Stack\Objects - TCPIP Demo App-C32\RSA.o
 .debug_abbrev  0x000050c0       0xab ..\Microchip\TCPIP Stack\Objects - TCPIP Demo App-C32\SSL.o
 .debug_abbrev  0x0000516b       0xab ..\Microchip\TCPIP Stack\Objects - TCPIP Demo App-C32\ARCFOUR.o
 .debug_abbrev  0x00005216       0xab ..\Microchip\TCPIP Stack\Objects - TCPIP Demo App-C32\BigInt.o
 .debug_abbrev  0x000052c1       0xab Objects - TCPIP Demo App-C32\CustomSSLCert.o

.debug_line     0x00000000     0x6cee
 *(.debug_line)
 .debug_line    0x00000000      0x3ad Objects - TCPIP Demo App-C32\MainDemo.o
 .debug_line    0x000003ad      0x5f8 Objects - TCPIP Demo App-C32\CustomHTTPApp.o
 .debug_line    0x000009a5       0x96 ..\Microchip\TCPIP Stack\Objects - TCPIP Demo App-C32\UDPPerformanceTest.o
 .debug_line    0x00000a3b      0x150 ..\Microchip\TCPIP Stack\Objects - TCPIP Demo App-C32\Announce.o
 .debug_line    0x00000b8b      0x168 ..\Microchip\TCPIP Stack\Objects - TCPIP Demo App-C32\ARP.o
 .debug_line    0x00000cf3       0xe3 ..\Microchip\TCPIP Stack\Objects - TCPIP Demo App-C32\Delay.o
 .debug_line    0x00000dd6      0x298 ..\Microchip\TCPIP Stack\Objects - TCPIP Demo App-C32\DHCP.o
 .debug_line    0x0000106e      0x1f8 ..\Microchip\TCPIP Stack\Objects - TCPIP Demo App-C32\DHCPs.o
 .debug_line    0x00001266      0x247 ..\Microchip\TCPIP Stack\Objects - TCPIP Demo App-C32\DNS.o
 .debug_line    0x000014ad      0x2b6 ..\Microchip\TCPIP Stack\Objects - TCPIP Demo App-C32\DynDNS.o
 .debug_line    0x00001763      0x4bf ..\Microchip\TCPIP Stack\Objects - TCPIP Demo App-C32\ENC28J60.o
 .debug_line    0x00001c22       0x96 ..\Microchip\TCPIP Stack\Objects - TCPIP Demo App-C32\FTP.o
 .debug_line    0x00001cb8      0x191 ..\Microchip\TCPIP Stack\Objects - TCPIP Demo App-C32\Hashes.o
 .debug_line    0x00001e49      0x29f ..\Microchip\TCPIP Stack\Objects - TCPIP Demo App-C32\Helpers.o
 .debug_line    0x000020e8      0x5c9 ..\Microchip\TCPIP Stack\Objects - TCPIP Demo App-C32\HTTP2.o
 .debug_line    0x000026b1       0x96 ..\Microchip\TCPIP Stack\Objects - TCPIP Demo App-C32\HTTP.o
 .debug_line    0x00002747      0x187 ..\Microchip\TCPIP Stack\Objects - TCPIP Demo App-C32\ICMP.o
 .debug_line    0x000028ce      0x144 ..\Microchip\TCPIP Stack\Objects - TCPIP Demo App-C32\IP.o
 .debug_line    0x00002a12      0x15e ..\Microchip\TCPIP Stack\Objects - TCPIP Demo App-C32\LCDBlocking.o
 .debug_line    0x00002b70      0x30d ..\Microchip\TCPIP Stack\Objects - TCPIP Demo App-C32\MPFS2.o
 .debug_line    0x00002e7d       0x96 ..\Microchip\TCPIP Stack\Objects - TCPIP Demo App-C32\MPFS.o
 .debug_line    0x00002f13      0x189 ..\Microchip\TCPIP Stack\Objects - TCPIP Demo App-C32\NBNS.o
 .debug_line    0x0000309c      0x12f ..\Microchip\TCPIP Stack\Objects - TCPIP Demo App-C32\Reboot.o
 .debug_line    0x000031cb      0x42e ..\Microchip\TCPIP Stack\Objects - TCPIP Demo App-C32\SMTP.o
 .debug_line    0x000035f9      0x76f ..\Microchip\TCPIP Stack\Objects - TCPIP Demo App-C32\SNMP.o
 .debug_line    0x00003d68      0x167 ..\Microchip\TCPIP Stack\Objects - TCPIP Demo App-C32\SNTP.o
 .debug_line    0x00003ecf      0x21b ..\Microchip\TCPIP Stack\Objects - TCPIP Demo App-C32\SPIEEPROM.o
 .debug_line    0x000040ea       0x96 ..\Microchip\TCPIP Stack\Objects - TCPIP Demo App-C32\SPIFlash.o
 .debug_line    0x00004180       0x96 ..\Microchip\TCPIP Stack\Objects - TCPIP Demo App-C32\SPIRAM.o
 .debug_line    0x00004216      0x163 ..\Microchip\TCPIP Stack\Objects - TCPIP Demo App-C32\StackTsk.o
 .debug_line    0x00004379      0x987 ..\Microchip\TCPIP Stack\Objects - TCPIP Demo App-C32\TCP.o
 .debug_line    0x00004d00      0x17b ..\Microchip\TCPIP Stack\Objects - TCPIP Demo App-C32\TCPPerformanceTest.o
 .debug_line    0x00004e7b      0x1cf ..\Microchip\TCPIP Stack\Objects - TCPIP Demo App-C32\Telnet.o
 .debug_line    0x0000504a       0x96 ..\Microchip\TCPIP Stack\Objects - TCPIP Demo App-C32\TFTPc.o
 .debug_line    0x000050e0      0x121 ..\Microchip\TCPIP Stack\Objects - TCPIP Demo App-C32\Tick.o
 .debug_line    0x00005201      0x198 ..\Microchip\TCPIP Stack\Objects - TCPIP Demo App-C32\UART2TCPBridge.o
 .debug_line    0x00005399       0xde ..\Microchip\TCPIP Stack\Objects - TCPIP Demo App-C32\UART.o
 .debug_line    0x00005477      0x23d ..\Microchip\TCPIP Stack\Objects - TCPIP Demo App-C32\UDP.o
 .debug_line    0x000056b4      0x30f Objects - TCPIP Demo App-C32\CustomSNMPApp.o
 .debug_line    0x000059c3      0x164 Objects - TCPIP Demo App-C32\UARTConfig.o
 .debug_line    0x00005b27      0x15c Objects - TCPIP Demo App-C32\GenericTCPClient.o
 .debug_line    0x00005c83      0x145 Objects - TCPIP Demo App-C32\GenericTCPServer.o
 .debug_line    0x00005dc8       0x96 Objects - TCPIP Demo App-C32\LegacyHTTPApp.o
 .debug_line    0x00005e5e      0x142 Objects - TCPIP Demo App-C32\PingDemo.o
 .debug_line    0x00005fa0      0x150 Objects - TCPIP Demo App-C32\SMTPDemo.o
 .debug_line    0x000060f0      0x30b ..\Microchip\TCPIP Stack\Objects - TCPIP Demo App-C32\BerkeleyAPI.o
 .debug_line    0x000063fb      0x189 Objects - TCPIP Demo App-C32\BerkeleyUDPClientDemo.o
 .debug_line    0x00006584      0x157 Objects - TCPIP Demo App-C32\BerkeleyTCPClientDemo.o
 .debug_line    0x000066db      0x163 Objects - TCPIP Demo App-C32\BerkeleyTCPServerDemo.o
 .debug_line    0x0000683e       0x96 ..\Microchip\TCPIP Stack\Objects - TCPIP Demo App-C32\ENCX24J600.o
 .debug_line    0x000068d4       0x96 Objects - TCPIP Demo App-C32\MPFSImg2.o
 .debug_line    0x0000696a       0x96 ..\Microchip\TCPIP Stack\Objects - TCPIP Demo App-C32\Random.o
 .debug_line    0x00006a00       0x96 ..\Microchip\TCPIP Stack\Objects - TCPIP Demo App-C32\RSA.o
 .debug_line    0x00006a96       0x96 ..\Microchip\TCPIP Stack\Objects - TCPIP Demo App-C32\SSL.o
 .debug_line    0x00006b2c       0x96 ..\Microchip\TCPIP Stack\Objects - TCPIP Demo App-C32\ARCFOUR.o
 .debug_line    0x00006bc2       0x96 ..\Microchip\TCPIP Stack\Objects - TCPIP Demo App-C32\BigInt.o
 .debug_line    0x00006c58       0x96 Objects - TCPIP Demo App-C32\CustomSSLCert.o

.debug_frame    0x00000000     0x2ccc
 *(.debug_frame)
 .debug_frame   0x00000000       0xec Objects - TCPIP Demo App-C32\MainDemo.o
 .debug_frame   0x000000ec      0x57c Objects - TCPIP Demo App-C32\CustomHTTPApp.o
 .debug_frame   0x00000668       0x50 ..\Microchip\TCPIP Stack\Objects - TCPIP Demo App-C32\Announce.o
 .debug_frame   0x000006b8       0xc8 ..\Microchip\TCPIP Stack\Objects - TCPIP Demo App-C32\ARP.o
 .debug_frame   0x00000780       0x4c ..\Microchip\TCPIP Stack\Objects - TCPIP Demo App-C32\Delay.o
 .debug_frame   0x000007cc       0xc8 ..\Microchip\TCPIP Stack\Objects - TCPIP Demo App-C32\DHCP.o
 .debug_frame   0x00000894       0x70 ..\Microchip\TCPIP Stack\Objects - TCPIP Demo App-C32\DHCPs.o
 .debug_frame   0x00000904       0xcc ..\Microchip\TCPIP Stack\Objects - TCPIP Demo App-C32\DNS.o
 .debug_frame   0x000009d0       0xc4 ..\Microchip\TCPIP Stack\Objects - TCPIP Demo App-C32\DynDNS.o
 .debug_frame   0x00000a94      0x3ec ..\Microchip\TCPIP Stack\Objects - TCPIP Demo App-C32\ENC28J60.o
 .debug_frame   0x00000e80       0xa8 ..\Microchip\TCPIP Stack\Objects - TCPIP Demo App-C32\Hashes.o
 .debug_frame   0x00000f28      0x1bc ..\Microchip\TCPIP Stack\Objects - TCPIP Demo App-C32\Helpers.o
 .debug_frame   0x000010e4      0x25c ..\Microchip\TCPIP Stack\Objects - TCPIP Demo App-C32\HTTP2.o
 .debug_frame   0x00001340       0xc8 ..\Microchip\TCPIP Stack\Objects - TCPIP Demo App-C32\ICMP.o
 .debug_frame   0x00001408       0x90 ..\Microchip\TCPIP Stack\Objects - TCPIP Demo App-C32\IP.o
 .debug_frame   0x00001498       0x8c ..\Microchip\TCPIP Stack\Objects - TCPIP Demo App-C32\LCDBlocking.o
 .debug_frame   0x00001524      0x2e4 ..\Microchip\TCPIP Stack\Objects - TCPIP Demo App-C32\MPFS2.o
 .debug_frame   0x00001808       0x70 ..\Microchip\TCPIP Stack\Objects - TCPIP Demo App-C32\NBNS.o
 .debug_frame   0x00001878       0x30 ..\Microchip\TCPIP Stack\Objects - TCPIP Demo App-C32\Reboot.o
 .debug_frame   0x000018a8      0x19c ..\Microchip\TCPIP Stack\Objects - TCPIP Demo App-C32\SMTP.o
 .debug_frame   0x00001a44      0x3e8 ..\Microchip\TCPIP Stack\Objects - TCPIP Demo App-C32\SNMP.o
 .debug_frame   0x00001e2c       0x50 ..\Microchip\TCPIP Stack\Objects - TCPIP Demo App-C32\SNTP.o
 .debug_frame   0x00001e7c      0x158 ..\Microchip\TCPIP Stack\Objects - TCPIP Demo App-C32\SPIEEPROM.o
 .debug_frame   0x00001fd4       0x70 ..\Microchip\TCPIP Stack\Objects - TCPIP Demo App-C32\StackTsk.o
 .debug_frame   0x00002044      0x3a0 ..\Microchip\TCPIP Stack\Objects - TCPIP Demo App-C32\TCP.o
 .debug_frame   0x000023e4       0x70 ..\Microchip\TCPIP Stack\Objects - TCPIP Demo App-C32\TCPPerformanceTest.o
 .debug_frame   0x00002454       0x34 ..\Microchip\TCPIP Stack\Objects - TCPIP Demo App-C32\Telnet.o
 .debug_frame   0x00002488       0xe4 ..\Microchip\TCPIP Stack\Objects - TCPIP Demo App-C32\Tick.o
 .debug_frame   0x0000256c       0xc0 ..\Microchip\TCPIP Stack\Objects - TCPIP Demo App-C32\UART2TCPBridge.o
 .debug_frame   0x0000262c       0x2c ..\Microchip\TCPIP Stack\Objects - TCPIP Demo App-C32\UART.o
 .debug_frame   0x00002658      0x228 ..\Microchip\TCPIP Stack\Objects - TCPIP Demo App-C32\UDP.o
 .debug_frame   0x00002880      0x128 Objects - TCPIP Demo App-C32\CustomSNMPApp.o
 .debug_frame   0x000029a8       0x30 Objects - TCPIP Demo App-C32\UARTConfig.o
 .debug_frame   0x000029d8       0x30 Objects - TCPIP Demo App-C32\GenericTCPClient.o
 .debug_frame   0x00002a08       0x30 Objects - TCPIP Demo App-C32\GenericTCPServer.o
 .debug_frame   0x00002a38       0x30 Objects - TCPIP Demo App-C32\PingDemo.o
 .debug_frame   0x00002a68       0x30 Objects - TCPIP Demo App-C32\SMTPDemo.o
 .debug_frame   0x00002a98      0x184 ..\Microchip\TCPIP Stack\Objects - TCPIP Demo App-C32\BerkeleyAPI.o
 .debug_frame   0x00002c1c       0x50 Objects - TCPIP Demo App-C32\BerkeleyUDPClientDemo.o
 .debug_frame   0x00002c6c       0x30 Objects - TCPIP Demo App-C32\BerkeleyTCPClientDemo.o
 .debug_frame   0x00002c9c       0x30 Objects - TCPIP Demo App-C32\BerkeleyTCPServerDemo.o

.debug_str      0x00000000      0x96a
 *(.debug_str)
 .debug_str     0x00000000       0x40 Objects - TCPIP Demo App-C32\MainDemo.o
 .debug_str     0x00000040       0x6d Objects - TCPIP Demo App-C32\CustomHTTPApp.o
 .debug_str     0x000000ad       0x12 ..\Microchip\TCPIP Stack\Objects - TCPIP Demo App-C32\UDPPerformanceTest.o
 .debug_str     0x000000bf       0x26 ..\Microchip\TCPIP Stack\Objects - TCPIP Demo App-C32\Announce.o
 .debug_str     0x000000e5       0x20 ..\Microchip\TCPIP Stack\Objects - TCPIP Demo App-C32\ARP.o
 .debug_str     0x00000105       0x12 ..\Microchip\TCPIP Stack\Objects - TCPIP Demo App-C32\Delay.o
 .debug_str     0x00000117       0x12 ..\Microchip\TCPIP Stack\Objects - TCPIP Demo App-C32\DHCP.o
 .debug_str     0x00000129       0x12 ..\Microchip\TCPIP Stack\Objects - TCPIP Demo App-C32\DHCPs.o
 .debug_str     0x0000013b       0x12 ..\Microchip\TCPIP Stack\Objects - TCPIP Demo App-C32\DNS.o
 .debug_str     0x0000014d       0x4b ..\Microchip\TCPIP Stack\Objects - TCPIP Demo App-C32\DynDNS.o
 .debug_str     0x00000198       0x7f ..\Microchip\TCPIP Stack\Objects - TCPIP Demo App-C32\ENC28J60.o
 .debug_str     0x00000217       0x12 ..\Microchip\TCPIP Stack\Objects - TCPIP Demo App-C32\FTP.o
 .debug_str     0x00000229       0x19 ..\Microchip\TCPIP Stack\Objects - TCPIP Demo App-C32\Hashes.o
 .debug_str     0x00000242       0x3c ..\Microchip\TCPIP Stack\Objects - TCPIP Demo App-C32\Helpers.o
 .debug_str     0x0000027e       0x2a ..\Microchip\TCPIP Stack\Objects - TCPIP Demo App-C32\HTTP2.o
 .debug_str     0x000002a8       0x12 ..\Microchip\TCPIP Stack\Objects - TCPIP Demo App-C32\HTTP.o
 .debug_str     0x000002ba       0x12 ..\Microchip\TCPIP Stack\Objects - TCPIP Demo App-C32\ICMP.o
 .debug_str     0x000002cc       0x1b ..\Microchip\TCPIP Stack\Objects - TCPIP Demo App-C32\IP.o
 .debug_str     0x000002e7       0x12 ..\Microchip\TCPIP Stack\Objects - TCPIP Demo App-C32\LCDBlocking.o
 .debug_str     0x000002f9       0x18 ..\Microchip\TCPIP Stack\Objects - TCPIP Demo App-C32\MPFS2.o
 .debug_str     0x00000311       0x12 ..\Microchip\TCPIP Stack\Objects - TCPIP Demo App-C32\MPFS.o
 .debug_str     0x00000323       0x1d ..\Microchip\TCPIP Stack\Objects - TCPIP Demo App-C32\NBNS.o
 .debug_str     0x00000340       0x12 ..\Microchip\TCPIP Stack\Objects - TCPIP Demo App-C32\Reboot.o
 .debug_str     0x00000352       0x5a ..\Microchip\TCPIP Stack\Objects - TCPIP Demo App-C32\SMTP.o
 .debug_str     0x000003ac      0x1b8 ..\Microchip\TCPIP Stack\Objects - TCPIP Demo App-C32\SNMP.o
 .debug_str     0x00000564       0x12 ..\Microchip\TCPIP Stack\Objects - TCPIP Demo App-C32\SNTP.o
 .debug_str     0x00000576       0x31 ..\Microchip\TCPIP Stack\Objects - TCPIP Demo App-C32\SPIEEPROM.o
 .debug_str     0x000005a7       0x12 ..\Microchip\TCPIP Stack\Objects - TCPIP Demo App-C32\SPIFlash.o
 .debug_str     0x000005b9       0x12 ..\Microchip\TCPIP Stack\Objects - TCPIP Demo App-C32\SPIRAM.o
 .debug_str     0x000005cb       0x12 ..\Microchip\TCPIP Stack\Objects - TCPIP Demo App-C32\StackTsk.o
 .debug_str     0x000005dd       0xa7 ..\Microchip\TCPIP Stack\Objects - TCPIP Demo App-C32\TCP.o
 .debug_str     0x00000684       0x27 ..\Microchip\TCPIP Stack\Objects - TCPIP Demo App-C32\TCPPerformanceTest.o
 .debug_str     0x000006ab       0x12 ..\Microchip\TCPIP Stack\Objects - TCPIP Demo App-C32\Telnet.o
 .debug_str     0x000006bd       0x12 ..\Microchip\TCPIP Stack\Objects - TCPIP Demo App-C32\TFTPc.o
 .debug_str     0x000006cf       0x12 ..\Microchip\TCPIP Stack\Objects - TCPIP Demo App-C32\Tick.o
 .debug_str     0x000006e1       0x12 ..\Microchip\TCPIP Stack\Objects - TCPIP Demo App-C32\UART2TCPBridge.o
 .debug_str     0x000006f3       0x12 ..\Microchip\TCPIP Stack\Objects - TCPIP Demo App-C32\UART.o
 .debug_str     0x00000705       0x48 ..\Microchip\TCPIP Stack\Objects - TCPIP Demo App-C32\UDP.o
 .debug_str     0x0000074d       0x61 Objects - TCPIP Demo App-C32\CustomSNMPApp.o
 .debug_str     0x000007ae       0x12 Objects - TCPIP Demo App-C32\UARTConfig.o
 .debug_str     0x000007c0       0x12 Objects - TCPIP Demo App-C32\GenericTCPClient.o
 .debug_str     0x000007d2       0x12 Objects - TCPIP Demo App-C32\GenericTCPServer.o
 .debug_str     0x000007e4       0x12 Objects - TCPIP Demo App-C32\LegacyHTTPApp.o
 .debug_str     0x000007f6       0x12 Objects - TCPIP Demo App-C32\PingDemo.o
 .debug_str     0x00000808       0x3d Objects - TCPIP Demo App-C32\SMTPDemo.o
 .debug_str     0x00000845       0x5f ..\Microchip\TCPIP Stack\Objects - TCPIP Demo App-C32\BerkeleyAPI.o
 .debug_str     0x000008a4       0x12 Objects - TCPIP Demo App-C32\BerkeleyUDPClientDemo.o
 .debug_str     0x000008b6       0x12 Objects - TCPIP Demo App-C32\BerkeleyTCPClientDemo.o
 .debug_str     0x000008c8       0x12 Objects - TCPIP Demo App-C32\BerkeleyTCPServerDemo.o
 .debug_str     0x000008da       0x12 ..\Microchip\TCPIP Stack\Objects - TCPIP Demo App-C32\ENCX24J600.o
 .debug_str     0x000008ec       0x12 Objects - TCPIP Demo App-C32\MPFSImg2.o
 .debug_str     0x000008fe       0x12 ..\Microchip\TCPIP Stack\Objects - TCPIP Demo App-C32\Random.o
 .debug_str     0x00000910       0x12 ..\Microchip\TCPIP Stack\Objects - TCPIP Demo App-C32\RSA.o
 .debug_str     0x00000922       0x12 ..\Microchip\TCPIP Stack\Objects - TCPIP Demo App-C32\SSL.o
 .debug_str     0x00000934       0x12 ..\Microchip\TCPIP Stack\Objects - TCPIP Demo App-C32\ARCFOUR.o
 .debug_str     0x00000946       0x12 ..\Microchip\TCPIP Stack\Objects - TCPIP Demo App-C32\BigInt.o
 .debug_str     0x00000958       0x12 Objects - TCPIP Demo App-C32\CustomSSLCert.o

.debug_loc
 *(.debug_loc)

.debug_macinfo
 *(.debug_macinfo)

.debug_weaknames
 *(.debug_weaknames)

.debug_funcnames
 *(.debug_funcnames)

.debug_typenames
 *(.debug_typenames)

.debug_varnames
 *(.debug_varnames)

/DISCARD/
 *(.note.GNU-stack)
OUTPUT(TCPIP Demo App-C32.elf elf32-tradlittlemips)

.mdebug.abi32   0x9d02f570        0x0

.rel.dyn        0x9d02f570        0x0
